:020000041000EA
:1000000000B5324B212058609868022188439860DF
:10001000D860186158612E4B002199600221596106
:100020000121F02299502B49196001219960352056
:1000300000F044F80222904214D00621196600F024
:1000400034F8196E01211966002018661A6600F04E
:100050002CF8196E196E196E052000F02FF8012189
:100060000842F9D1002199601B49196000215960AB
:100070001A491B48016001219960EB211966A021F2
:10008000196600F012F800219960164914480160C1
:100090000121996001BC002800D000471248134993
:1000A000086003C880F30888084703B5996A0420EC
:1000B0000142FBD001200142F8D103BD02B5186610
:1000C0001866FFF7F2FF186E186E02BD00000240BE
:1000D000000000180000070000035F00212200005C
:1000E000F4000018222000A00001001008ED00E03C
:1000F00000000000000000000000000074B24E7A12
:1001000000200420F7010010C3010010C5010010F9
:10011000C1010010C1010010C1010010C101001097
:10012000C1010010C1010010C1010010C701001081
:10013000C1010010C1010010C9010010CB01001065
:10014000CD010010CD010010CD010010CD01001037
:10015000CD010010CD010010CD010010CD01001027
:10016000CD010010CD010010CD010010CD01001017
:10017000CD010010CD010010CD010010CD01001007
:10018000CD010010CD010010CD010010CD010010F7
:10019000CD010010CD010010CD010010CD010010E7
:1001A000CD010010CD010010CD010010CD010010D7
:1001B000CD010010CD010010CD010010CD010010C7
:1001C00000BE00BE00BE00BE00BE00BE00F04BF888
:1001D000103800BEF2EB887174AE001098AE0010BB
:1001E0003402001090A31AE700202149086006C8D5
:1001F00081F3088810471F48006800282FD10DA4FC
:100200000ECC002902D000F012F8F9E71A491B4A77
:10021000002000E001C19142FCD1194988471949E9
:1002200088471949884700BEFDE701C901C29A42C3
:10023000FBD3704798AE0010C00000204805002096
:1002400020B30010000004200000042020B30010A0
:1002500000100420001004200000000070470B482C
:1002600004F02AFF0047EFF30580C0B2704700009A
:1002700008ED00E0000000D000800020A48E0220E5
:10028000E5350010351F0010A1350010575600004D
:1002900006005250ABB3605354A5001006005250F4
:1002A000861C030264A50010060052505422A29D31
:1002B00074A5001005005250DE65F46820B30010EC
:1002C000F8B5C04610B5064C2378002B07D1054B76
:1002D000002B02D0044800E000BF0123237010BDB2
:1002E0000881022000000000B8940010044B10B5F3
:1002F000002B03D00349044800E000BF10BDC046F6
:10030000000000000C810220B894001070B5984BDA
:100310001A6801239340A020C005964943509301D9
:10032000A021C9058C466344DB68DB01F7D4924BFE
:100330001A680123934008008E4943509301A0217D
:10034000C9058C466344DB68DB01F7D48B4B1A6824
:10035000012393400800874943509301A021C90518
:100360008C466344DB68DB01F7D4854B19680123B5
:100370008B4060467F4A83508B01A022D205944671
:100380006344DA6880235B0414001C401A42F3D1F2
:100390007C4D2A68303280239B01134301221A606E
:1003A0000021072003F02EFB2A68774B18680430E1
:1003B000764B9A4200D008240019002103F022FB5A
:1003C0007349072003F060FB694B1A68714B0C2AD4
:1003D00000D9ADE070490B40D20213430C22934385
:1003E000043A13436D4A13406D4A13406D4A13405B
:1003F000012213436C490B4093435D4A106882010C
:10040000A021C9058C4662440021116051609160B1
:10041000136108F0C1FD584B1A685E4B0C2A00D9D5
:100420008CE05D490B40D20213430C229343043A03
:1004300013435A4A13405A4A13405A4A134001225E
:10044000134359490B4093434B4A10688201A02142
:10045000C9058C46624400211160516091601361AE
:1004600008F09AFD454B1A684A4B0C2A00D96BE0FC
:1004700049490B40D20213430C229343043A1343DD
:10048000464A1340464A1340464A1340012213434A
:1004900045490B409343394A10688201A021C905A0
:1004A0008C4662440021116051609160136108F034
:1004B00073FD334B1A68374B0C2A4BD836490B4027
:1004C000D20213430C229343043A1343334A13409A
:1004D000334A1340334A134001242343324A134022
:1004E000A343274A10688201A021C9058C466244B3
:1004F0000021116051609160136108F04DFD214BA6
:100500001868214B196803688C40A343036008F006
:10051000F3FD264B1B78002B22D0254B1A68194B74
:100520001868244908F032FE234B01221A7070BD6E
:10053000224B234AC021234803F036F81F4B204AA0
:10054000C021204803F030F81C4B1D4AC0211D4833
:1005500003F02AF8194B1A4AC0211A4803F024F86C
:10056000134B1A68074B1868174908F00FFEDBE7B2
:100570006C870220440400007087022074870220E8
:1005800078870220D4860220548E0220000020505A
:100590000D03001010801F00FF87FFFF3FF8FFFFD3
:1005A000FFFFBFFFFFFFDFFFFFFF7FFF9D8E0220EA
:1005B000D086022010960010948E0220B89400106D
:1005C00030960010D8940010F095001070B59D4B37
:1005D0001A6801239340A020C0059B494350930112
:1005E000A021C9058C466344DB68DB01F7D4974B37
:1005F0001A68012393400800934943509301A021B6
:10060000C9058C466344DB68DB01F7D4904B1A685C
:100610000123934008008C4943509301A021C90550
:100620008C466344DB68DB01F7D48A4B19680123ED
:100630008B406046844A83508B01A022D2059446A9
:100640006344DA6880235B0414001C401A42F3D12F
:10065000814D2A68303280239B01134301221A60A6
:100660000021072003F0CEF92A687C4B186804307B
:100670007B4B9A4200D008240019002103F0C2F9F4
:100680007849072003F000FA6E4B1A68764B0C2A63
:1006900000D9BEE075490B40D20213430C229343AC
:1006A000043A1343724A1340724A1340724A134089
:1006B0000122134371490B409343624A106882013F
:1006C000A021C9058C4662440021116051609160EF
:1006D000136108F061FC5D4B1A68634B0C2A00D96A
:1006E0009DE062490B40D20213430C229343043A2B
:1006F00013435F4A13405F4A13405F4A134001228D
:1007000013435E490B409343504A10688201A02175
:10071000C9058C46624400211160516091601361EB
:1007200008F03AFC4A4B1A684F4B0C2A00D97CE07F
:100730004E490B40D20213430C229343043A134315
:100740004B4A13404B4A13404B4A13400122134378
:100750004A490B4093433E4A10688201A021C905D3
:100760008C4662440021116051609160136108F071
:1007700013FC384B1A683C4B0C2A5CD83B490B40A5
:10078000D20213430C229343043A1343384A1340D2
:10079000384A1340384A134001242343374A134050
:1007A000A3432C4A10688201A021C9058C466244EB
:1007B0000021116051609160136108F0EDFB264D3E
:1007C0002868264B1968036822008A409343036017
:1007D00008F092FC2A4B1A6828682A4908F0D6FCCF
:1007E000294D2868294E0368220031688A409343C6
:1007F0000360002208F014FD3168286808F07CFCD2
:10080000234B1A682868234908F0C0FC224B1C704F
:1008100070BD224B224AC021224802F0C5FE1F4B68
:100820001F4AC0211F4802F0BFFE1C4B1C4AC021BA
:100830001C4802F0B9FE194B194AC021194802F0B0
:10084000B3FEC0466C87022044040000708702207B
:100850007487022078870220D4860220548E0220DA
:1008600000002050CD05001010801F00FF87FFFF03
:100870003FF8FFFFFFFFBFFFFFFFDFFFFFFF7FFF2F
:10088000D0860220D0950010788E0220588E02204B
:10089000748E02203C040020948E0220B894001034
:1008A00030960010D894001070B59C4B1A68012344
:1008B0009340A020C0059A4943509301A021C90547
:1008C0008C466344DB68DB01F7D4964B1A6801233E
:1008D00093400800924943509301A021C9058C46DA
:1008E0006344DB68DB01F7D48F4B1A680123934024
:1008F00008008B4943509301A021C9058C466344ED
:10090000DB68DB01F7D4894B196801238B40604613
:10091000834A83508B01A022D20594466344DA684F
:1009200080235B0414001C401A42F3D1804D2A68D6
:10093000303280239B01134301221A6000210720DB
:1009400003F060F82A687B4B186804307A4B9A42AF
:1009500000D008240019002103F054F8774907203B
:1009600003F092F86D4B1A68754B0C2A00D9BDE064
:1009700074490B40D20213430C229343043A1343AD
:10098000714A1340714A1340714A134001221343C4
:1009900070490B409343614A10688201A021C90548
:1009A0008C4662440021116051609160136108F02F
:1009B000F3FA5C4B1A68624B0C2A00D99CE061493F
:1009C0000B40D20213430C229343043A13435E4A72
:1009D00013405E4A13405E4A1340012213435D49AF
:1009E0000B4093434F4A10688201A021C9058C46F1
:1009F00062440021116051609160136108F0CCFAEB
:100A0000494B1A684E4B0C2A00D97BE04D490B40EC
:100A1000D20213430C229343043A13434A4A13402D
:100A20004A4A13404A4A13400122134349490B40A2
:100A300093433D4A10688201A021C9058C46624457
:100A40000021116051609160136108F0A5FA374BE5
:100A50001A683B4B0C2A5BD83A490B40D20213432D
:100A60000C229343043A1343374A1340374A134046
:100A7000374A134001242343364A1340A3432B4AE9
:100A800010688201A021C9058C46624400211160D2
:100A900051609160136108F07FFA254D2868254B5D
:100AA0001968036822008A409343036008F024FB1E
:100AB000294B1A682949286808F068FB2868284EDD
:100AC0000368220031688A4093430360002208F0E3
:100AD000A7FB3168286808F00FFB224B1A682868CA
:100AE000214908F053FB214B1C7070BD204B214A5B
:100AF000C021214802F058FD1D4B1E4AC0211E484E
:100B000002F052FD1A4B1B4AC0211B4802F04CFD5B
:100B1000174B184AC021184802F046FD6C87022086
:100B20004404000070870220748702207887022026
:100B3000D4860220548E022000002050A908001004
:100B400010801F00FF87FFFF3FF8FFFFFFFFBFFF81
:100B5000FFFFDFFFFFFF7FFFD0860220B095001070
:100B6000588E0220748E022020040020948E0220D1
:100B7000B894001030960010D894001070B504009E
:100B800001238B40DDB2013DEDB2FF20002307E0E1
:100B90008021490119435A00084E91530133DBB2B9
:100BA0001F2B09D82A001A40A242F1D05A0003494B
:100BB000034850521800F1E770BDC046248102205E
:100BC000A0A0FFFFF8B5012008F0EEF9C84C2060A6
:100BD000012008F0E9F9C74B1860012008F0E4F99A
:100BE000C54B1860012008F0DFF9C44B186021687C
:100BF000C34A0C2900D92AE1C24B1A40C9020A4350
:100C00000C20824308210A43BF4B1A40BF4B1A40B5
:100C1000BF4B1A4001231A43BE4B1A4010239A437C
:100C200013002022134383430B43B24A12680C2A59
:100C300000D912E1B3491940D3020B43B64A1068F8
:100C4000B64A12680432B649884200D10BE1082145
:100C500052183F2A00D908E1B2491940D3030B4387
:100C6000A94A1340F822D2001343A24A1068A449AB
:100C70000C2800D9FFE0A34A1140C00201430C2414
:100C8000A14308200143A04A1140A04A1140A04AB4
:100C90001140012211439F4A1140102291430A0042
:100CA00020210A43A2430243934909680C2900D931
:100CB000E7E094481040CA02024397490C689749FC
:100CC000096804319648844200D1E0E00820091800
:100CD0003F2900D9DDE093481040CA0302438A4906
:100CE0000A40F821C9000A4383490C6884480C2C47
:100CF00000D9D4E083490840E40220430C25A843EE
:100D00000824204380490840804908408049084021
:100D1000012108437F490840102188430100202019
:100D20000143A9432143754800680C2800D9BCE061
:100D3000744C0C40C102214377480568774800682D
:100D40000430774CA54200D1B5E0082400193F28B3
:100D500000D9B2E0734C0C40C10321436A48014002
:100D6000F820C000014365480568654C0C2D00D98A
:100D7000A9E064480440ED022C430C26B443082546
:100D80002C4361480440614804406148044001200C
:100D90000443604804401020844320002024204362
:100DA000B0432843524C24680C2C00D991E0554D97
:100DB0000540E0022843584C2668584C2468043407
:100DC000574DAE4200D18AE0082564193F2C00D966
:100DD00087E0544D0540E00328434B4C2040F82465
:100DE000E4002043454C27684B4C26684B4C246854
:100DF0000834A5007519BF01A024E405A446674482
:100E00003D60494C7C608026B601BE6038613A483E
:100E10000068800160440560444FE71947608660C0
:100E2000016134490968890161440D604048201816
:100E300048608E600A612E4A126892016244156011
:100E40003C498C46644454609660D360F8BD3A4B8C
:100E50003A4AC0213A4802F0A7FB374B374AB8312B
:100E6000374802F0A1FB0021F2E6364B364AB221A8
:100E7000334802F099FB304B304AC021304802F031
:100E800093FB2D4B2D4AC0212D4802F08DFB0020F5
:100E90001DE72C4B2C4AB221294802F085FB264B3A
:100EA000264AC021264802F07FFB234B234AC0215B
:100EB000234802F079FB002448E7224B224AB22162
:100EC0001F4802F071FB1C4B1C4AC0211C4802F059
:100ED0006BFB194B194AC021194802F065FB00252C
:100EE00073E7184B184AB221154802F05DFBC04663
:100EF0006C87022070870220748702207887022086
:100F000010801F00FF87FFFF3FF8FFFFFFFFBFFFBD
:100F1000FFFFDFFFFFFF7FFFD4860220548E0220F9
:100F200000002050FF7FE0FF000002200080FFFF54
:100F30000000FFFF0080FEFFB89400103096001004
:100F4000D8940010249500104C960010F0B5DE46A1
:100F500057464E464546E0B597B003900D00140045
:100F6000049320AB1E7821AB1A78934622AB1F78EE
:100F700023AB1A8890460A1980231B029A4200D399
:100F80000AE23D4B984200D90EE2182E00D90DE23C
:100F90005A460F2A00D90BE2052F00D90AE2002F8A
:100FA00000D109E2BB18102B01DD0020F5E1802201
:100FB00092020021314805F02DF8314B1D60314B74
:100FC0001C60314B1E70314B01221A7000230498B3
:100FD00006E0C25C2E49895C2E4AD1540133DBB253
:100FE000B342F6D32A4B5A469B5C1A0004932A4B11
:100FF0001A70052002F08CFC04F03CFF8146039B34
:10100000580004F037FF011C484604F014FF8146E5
:10101000224D234B1D60280008F0E4F8214B9B462D
:101020002148186008F0DEF85B461B68AB420ED022
:101030000721002001F098F8194B1A68174B9A42C3
:1010400007D00721012001F08FF8002508E00621D4
:10105000EFE70621F6E7062101F086F80135EDB24B
:10106000B54223D20E4B1A680A4B585D0B4B9A427D
:10107000F1D00721F0E7C04600E1F505008000202F
:10108000A08B02209C8B02209C8E02209B8E022033
:1010900064960010848B02209F8E02200000205056
:1010A000D4860220788E022000003050C34D0121EA
:1010B000286808F031F80200C14B9A461860286889
:1010C00053009B18DB00D033C318802149010B4328
:1010D00080210906196019600368043201219140DA
:1010E0000B430360B74908F035F8B74B9B461860CF
:1010F000534619682868002300931D33022208F024
:10110000C9F85B461B689A46102200210AA804F021
:1011100081FF80256D020A95F8235B020B938023E3
:10112000DB020C93C0231B030C9310220AA906A810
:1011300004F076FF5346191D5A1D079B0393A34BDA
:1011400003980340C9010B43120313430793102272
:1011500006A90EA804F064FF119B03939C4B039A0D
:1011600013401D431195484604F0ACFE85B2002D96
:1011700000D10DE1280004F07DFE011C484604F07A
:1011800050FE8721C90504F06CFE04F09BFEC3B23B
:101190001B022D041D430E95109B03938D4A1A408C
:1011A0008D4B134310930F9B03938C4A1A4080235B
:1011B0005B0413430F93814D2A6811003031802363
:1011C0009B011943012008602D32FF321343802216
:1011D00052001A608249063002F02CFC01210720DF
:1011E00002F010FC2A68764B186804307D4B9A4256
:1011F00000D1CFE00823C018012102F003FC724B9C
:101200001A686F4B9A466D4B9B460EAB5146096868
:101210005846006808F076F8734D0121286807F0F9
:101220007BFF724B994618602A6843001B18DB004D
:10123000D033D318802149010B438021090619605E
:10124000196013680430012181400B431360434649
:10125000D8B23900FFF792FC05906549286807F07D
:1012600079FF644B984618604B461968286801233B
:101270000093002208F00EF84B46196828680023F6
:1012800000933B00049E320008F004F843461F68B8
:10129000102200210AA804F0BDFE80256D020A95E7
:1012A000F8235B020B938023DB020C93C0231B0308
:1012B0000C9310220AA906A804F0B2FE3B001F33CB
:1012C0001A00079B0393414B03990B40FF013B43DB
:1012D00012031343079309990391CA00D20880218E
:1012E00089050A430992444A13400793102206A92C
:1012F00012A804F095FE102212A90EA804F090FE88
:10130000119B0393324B03990B40F6031E43119636
:101310003A4B1E408023DB041E431196384B1E407F
:1013200011960E95FFF74EFC5B461A6853461D68F2
:1013300011680123AB4099430B431360013C516892
:1013400028001030012383400B42F8D1291D890069
:101350008C5051680B42FCD10435AD0001235B4237
:10136000AB50224C204D0EAB059A2168286807F03F
:10137000C9FF296820680A68012383409A43134300
:101380000B6000231F4A13701F4A1370012004E0F2
:101390000023FDE600232EE7002017B0F0BCBB467B
:1013A000B246A946A046F0BD0020F6E70020F4E7CB
:1013B0000020F2E70020F0E70020EEE7D4860220CC
:1013C000548E0220D0950010D08602207F00FEFFB0
:1013D000FF7FF0FFFFFF0AFE0000D101FFFFFFE0EB
:1013E000CD05001000002050788E0220588E02207B
:1013F0003C040020748E0220FFFFFF9F1FFCFFE3D0
:10140000FF83FFFF948E0220958E0220F0B5DE460A
:1014100057464E464546E0B595B002900D00140083
:1014200003931EAB1E781FAB1A78934620AB1F7830
:1014300021AB1A8890460A1980231B029A4200D3D6
:10144000FEE13A4B984200D902E2182E00D901E29F
:101450005A460F2A00D9FFE1102F00D9FEE1002FD4
:1014600000D1FDE1BB18102B01DD0020E9E1802255
:10147000920200212E4804F0CDFD2E4B1D602E4B14
:101480001C602E4B1E702E4B01221A7000230398F5
:1014900006E0C25C2B49895C2B4AD1540133DBB294
:1014A000B342F6D3274B5A469B5C1A000393274B53
:1014B0001A70052002F02CFA04F0DCFC8146029B35
:1014C000580004F0D7FC011C484604F0B4FC8146E7
:1014D0001F4B9B461F4D1D60280007F083FE5B4697
:1014E0001B68AB420ED00721002000F03DFE184BD8
:1014F0001A68184B9A4207D00721012000F034FEE9
:10150000002508E00621EFE70621F6E7062100F0B6
:101510002BFE0135EDB2B5421ED20D4B1A680A4BB7
:10152000585D0C4B9A42F1D00721F0E700E1F50538
:1015300000800020A08B02209C8B02209C8E022029
:101540009B8E022064960010848B02209F8E0220C6
:10155000D486022000002050C24D0121286807F0E7
:10156000DBFD0200C04B9A461860286853009B18A8
:10157000DB00D033C318802149010B4380210906C9
:101580001960196003680432012191400B43036024
:10159000B64907F0DFFDB64B9B4618605346196805
:1015A0002868002300931D33022207F073FE5B4678
:1015B0001B689A461022002108A804F02BFD802504
:1015C0006D020895F8235B0209938023DB020A93DE
:1015D000C0231B030A93102208A904A804F020FDCD
:1015E0005346591D9A1D059B0293A24B0298034036
:1015F000C9010B43120313430593102204A90CA83D
:1016000004F00EFD0F9B02939B4B029A13401D4367
:101610000F95484604F056FC85B2002D00D10BE131
:10162000280004F027FC011C484604F0FAFB87213F
:10163000C90504F016FC04F045FCC3B21B022D04DE
:101640001D430C950E9B02938C4A1A408C4B1343FE
:101650000E930D9B02938B4A1A4080235B04134325
:101660000D93804D2A681100303180239B0119436E
:10167000012008602D32FF321343802252001A608D
:101680008149063002F0D6F90121072002F0BAF9AB
:101690002A68754B186804307C4B9A4200D1CDE023
:1016A0000823C018012102F0ADF9714B1A686E4B86
:1016B0009A466C4D0CAB51460968286807F022FE2B
:1016C0000121286807F028FD0200714B9946186037
:1016D000286853009B18DB00D033C31880214901D0
:1016E0000B43802109061960196003680432012147
:1016F00091400B430360674B3B43674A5381674903
:1017000007F028FD664B9B4618604B461968286811
:1017100001230093002207F0BDFD4B46196828689D
:10172000002300933B00039E320007F0B3FD5B46AD
:101730001F681022002108A804F06CFC80235B02C3
:101740009B460893F8235B0209938023DB020A93EC
:10175000C0231B030A93102208A904A804F060FC0C
:101760003B0008331A00059B0293424B02990B4041
:10177000F9010B43120313430593102204A910A887
:1017800004F04EFC102210A90CA804F049FC0F9B99
:101790000293394B02990B40F6031E430F96414BBF
:1017A0001E408023DB041E430F965B460C930E9B6A
:1017B0000293324B029A13400E934B4619680CABBE
:1017C0003A00286807F09EFDFFF7FCF92A685346A7
:1017D0001D6811680123AB4099430B431360013C22
:1017E000516828001030012383400B42F8D1291D95
:1017F00089008C5051680B42FCD10435AD000123A7
:101800005B42AB50224B1C6811680123A3409943F3
:101810000B431360516820001030012383400B42BA
:10182000F8D10434A4004346A35000231E4A137089
:101830001E4A1370012004E00023FFE6002330E776
:10184000002015B0F0BCBB46B246A946A046F0BD8C
:101850000020F6E70020F4E70020F2E70020F0E7A0
:101860000020EEE7D4860220548E0220B0950010AE
:10187000D08602207F00FEFFFF7FF0FFFFFF0AFE01
:101880000000D101FFFFFFE0A90800100000205078
:10189000588E022040600000280400202004002010
:1018A000748E02201FFCFFE3948E0220958E02208E
:1018B000F0B5D6464F464646C0B590B082460F00BA
:1018C00016001C0018AB1D7819AB1B7899461AAB93
:1018D0001B7898468A1880231B029A4200D368E13D
:1018E000B84B984200D96BE1182D01D9002061E175
:1018F000802292020021B44804F08CFBB34B1F609D
:10190000B34B1E60B34B1D70B34B42461A70B34BC2
:1019100000221A70002106E0635CB14AD25CB14B30
:101920005A540131C9B2A942F6D3AD4B4A469B5C29
:101930009946AD4B4A461A70052001F0E9FF04F0C4
:1019400099FA041C5346580004F094FA011C201C18
:1019500004F071FA071CA54CA548206007F042FC72
:101960000121206807F0D8FB0200A24B1860206814
:1019700053009B18DB00D033C318802149010B436F
:101980008021090619601960036804320121914021
:101990000B4303604346002B18D0974907F0DAFB4E
:1019A000964B1860934B1968904C20680023009365
:1019B0002033002207F06EFC22688D4B9A420BD038
:1019C0000721484600F0D0FB00240CE08C4907F0CA
:1019D000C1FB8A4B1860E5E70621F2E7062100F01B
:1019E000C3FB0134E4B2AC4208D2804B1A687D4B91
:1019F000185D7F4B9A42F1D00721F0E74346002B58
:101A000000D1A8E07D4B1C681022002108A804F03A
:101A100001FB80235B020893F8235B020993802378
:101A2000DB020A93C0231B030A93102208A904A80F
:101A300004F0F6FA22000A32059B0393714B0399D6
:101A40000B40E4012343120313430593102204A91E
:101A50000CA804F0E5FA0F9B03936B4B039A134019
:101A60000F93381C04F02EFA84B2002C00D19CE0B5
:101A7000200004F0FFF9011C381C04F0D2F9872182
:101A8000C90504F0EEF904F01DFAC0B20002240406
:101A900004430C940E9B03935C4A1A40A023DB0280
:101AA00013430E930D9B0393594B039A13404A46DD
:101AB000120613430D934D4C2268110030318023E0
:101AC0009B011943012008602D32FF32134380220D
:101AD00052001A604F49063001F0ACFF0121072087
:101AE00001F090FF2268434B18680430404B9A4243
:101AF0005DD00823C018012101F084FF3F4B1A6814
:101B00003C4C3A4D0CAB2168286807F0FBFBFFF713
:101B100059F8296825680A680123AB409A431343A2
:101B20000B60013E48682C0010340123A34003429F
:101B3000F8D12A1D920056504A681342FCD1043550
:101B4000AD0001235B426B500023334A1370334ACC
:101B5000137001202EE0294B1C681022002108A8D8
:101B600004F058FA80235B020893F8235B02099380
:101B70008023DB020A93C0231B030A93102208A9C7
:101B800004A804F04DFA221D0534059B03931D4B58
:101B900003990B40D20113432403234305931022DE
:101BA00004A90CA804F03CFA55E700206EE70023D6
:101BB000A0E7002010B0E0BCBA46B146A846F0BD90
:101BC0000020F7E700E1F50500800020A08B02204F
:101BD0009C8B02209C8E02209D8E02209B8E0220D8
:101BE00064960010848B02209E8E0220D4860220F0
:101BF00000002050548E0220F0950010D086022064
:101C0000109600107F00FEFFFF7FF0FFFFFF0AFE2F
:101C1000FFFFFFE00D030010948E0220958E02203E
:101C2000024B187801235840C0B27047948E0220AE
:101C3000F0B5CE46474680B580468C46434B1B7870
:101C4000002B10D0424B1B68424A12689B18424638
:101C50001360414B62461B6813604048C0BCB946E4
:101C6000B046F0BD01338022120293421CDA9A0082
:101C70003A4C12590132F5D1013B17D4344A156858
:101C8000344A1268AD186A1E9A4211D95B1B344A55
:101C900091464B44304A13602F4B1C68314B1B78E4
:101CA000002B2CD1002143E00023E7E72C4BE5E794
:101CB0005B1B0133284A1360EEE72B4B9A5D023A17
:101CC000012393400340921BD3401F430136274B0F
:101CD0001B78B342F1DC631CA400204AA750802289
:101CE0001202934209D21C0001318D422AD9A3006D
:101CF0001A4A985800260027E9E70024F4E7002153
:101D0000F3E7194B9E5C0123B3400340B61AF3403E
:101D10001F430132154B1B789342F2DC631CA40075
:101D20000E4AA75080221202934209D21C000131B0
:101D30008D4207D9A300094A985800220027E9E7F5
:101D40000024F4E7014B01221A707BE7958E0220F4
:101D5000A08B02209C8B0220A48B022000800020FC
:101D6000FF7F00009B8E0220848B02209C8E02202D
:101D700070B584B0002004F0F5FA431C1FD063490D
:101D80000A78531CDBB20B7061498854012B10D0C8
:101D9000022B16D0022B12D91C009A1E5C498A5CB9
:101DA000AA2A0CD15A1E8A5C552A08D10022002189
:101DB00018E00A78552AEBD0544B00221A7004B070
:101DC00070BD534A5278AA2AE4D0504B00221A70B0
:101DD000F5E701324E4DAE5C0138FF387040685473
:101DE00001310132944206DD4948805CF028F0D090
:101DF000474D6854F4E7464A9278002A08D0012AF1
:101E000010D0444804F06CFA404B00221A70D6E718
:101E1000052B03D03F4804F063FAF5E73E4804F091
:101E20005FFAF1E73D4B3E4A13601B78012B27D048
:101E3000022B46D0364C6579230009332B22A15C56
:101E4000E26A12020A432721605CA16A0902014387
:101E50002320265C606A000230436E1EB541029565
:101E6000257901952125645D0094FFF721FD002867
:101E700048D02C4804F034FA2B4B01221A70C3E7E7
:101E80002A4B1C00093C2B22A15CE26A12020A4385
:101E90002721605CA16A090201432320255C606A56
:101EA00000022843E679257A2D02354303956579AA
:101EB0000295257901952125645D0094FFF7A6FA26
:101EC000D5E71A4B1C00093C2B22A15CE26A1202E6
:101ED0000A432721605CA16A090201432320255C93
:101EE000606A00022843E679257A2D02354303957E
:101EF00065790295257901952125645D0094FFF7A8
:101F000025F8B4E70A4804F0EBF97DE7938E022048
:101F1000AC8B02203895001048950010AF8B022042
:101F2000408C02205C950010968E0220B58B02201A
:101F30006C95001030B585B003AB02AA01A93C48EE
:101F400000F0BAF8002803D139493A4801F0C6FB3D
:101F5000039A0299019800F073F804F0FFF9FA204F
:101F6000800000F017FF80220021334804F052F86F
:101F7000192000F011F9D0231B06802292045A6226
:101F800019E00134029B9C420DD2039B5A1C039220
:101F9000E85C04F071F980239B02039A9A42F0D323
:101FA00000230393EDE7254B00221A70D0231B0674
:101FB000802292049A61D0231B06802292045A61E7
:101FC0001E4B1B78002B30D0FFF72AFE00281FD1B4
:101FD00002AC03A92000FFF72BFE0500642000F0EF
:101FE000D9FE207804F048F9607804F045F9A0782B
:101FF00004F042F9E07804F03FF9642000F0CAFEF2
:10200000029B9B000293039B9B0003930024B9E770
:10201000D02424068025AD04A561642000F0BAFE1A
:102020006561642000F0B6FEC0E7FFF7A1FEBDE7E2
:10203000400D03007C950010AC8B0220968E022090
:10204000F0B583B004000D00160000F029F9002857
:1020500001D003B0F0BD154F00973B0001220121D4
:10206000053001F053FB00962B002200012110489F
:1020700001F064FE31006943200003F071F80400B0
:102080000C4B009300220221042001F03FFB00943E
:10209000230000220121052001F038FB00973B00BE
:1020A00002220021062001F031FBD2E7006CDC02A5
:1020B00000800240001BB700F0B5DE4657464E4692
:1020C0004546E0B583B080468B46009201930420DC
:1020D00001F01EFCFA21890003F042F88246A02399
:1020E0005B0099462CE0013C002C20D025007D436C
:1020F0002900300003F034F84045F4D129003000C5
:1021000003F02EF80029EED173019B1B9B009E1952
:10211000F6005B461E60009B1F60019B1C60012057
:1021200003B0F0BCBB46B246A946A046F0BD013F95
:10213000002F01D03C00D7E701235B429C46E144DD
:102140004B460F2B09D956464B465E43044BF218BB
:10215000044B9A42F0D80727EAE70020E0E7C046A0
:1021600080E5F9FF804F120010B58300084A9446BD
:1021700063441C6840226240C02414408022520103
:1021800013431C60C000034B9C466044416010BD7B
:1021900004C001400040014010B501238340D0221B
:1021A0001206936293610521FFF7DEFF10BD000068
:1021B000EFF3108072B6034B1B68002BFBD0BFF30C
:1021C0005F8F70472C0100D0BFF35F8F024B00225E
:1021D0001A6080F3108870472C0100D0F8B5060013
:1021E0000C001500FFF7E4FFE308F718F15C072285
:1021F0002240012393400B4205D1DBB20B433B70DD
:10220000FFF7E2FFF8BD2100280001F067FAF0B502
:1022100083B00600019114001F00FFF7C9FF00E022
:102220000134BC420CD8E308F518F35C07212140C7
:1022300001228A401A42F3D1D2B21A432A7001E035
:1022400001246442FFF7C0FF002C02DB200003B032
:10225000F0BD019B002BF9D0089801F03FFA000077
:1022600070B505000C00FFF7A3FFE308EE18EA5C69
:1022700007210C400123A340134204D09A4332703B
:10228000FFF7A2FF70BD034B034A2C31034801F056
:102290008BF9C0467C960010DC9600109C960010CE
:1022A000034B1B6802201840431E9841C0B2704780
:1022B00000C00640002307E0054A9A189200BFF3C9
:1022C0005F8F0021116001331F2BF5D97047C04685
:1022D00040000034054A1078431CDBB21370172B02
:1022E00002D9130010221A707047C0464204002021
:1022F00000B583B00100044B00931F23182203484C
:10230000FFF785FF03B000BDEC960010D8860220D1
:1023100070B505000C00080000F0CCFD200000F0B6
:10232000D5FE0849200000F015FEFFF7D3FF064B4D
:102330009C466044800068602C75A400034BE55007
:1023400070BDC0465526001040000034308C02207D
:102350000A4B1A68EFF3108172B61368002BFCD099
:10236000BFF35F8F054B1B68BFF35F8F00221A60BE
:1023700081F3108840BF002000217047508E02205A
:1023800010B5002922D003681B7B99421ED8174B39
:102390009C466144090183689C4661440C68496815
:1023A000002A19D003681B7B9A4215D883680F480E
:1023B0008446624412019A18106853680200012092
:1023C0008B4201D80ED00020C0B210BD084B094A84
:1023D0003B21094801F0E8F8054B064A3B21064835
:1023E00001F0E2F8A242EFD8EDE7C046FFFFFF0F91
:1023F00054970010109A00101C97001010B5002977
:102400001ED0037B99421BD84B005B18033B04682A
:10241000A4466344002919D0002A1DD0914221D03E
:10242000002A25D0047BA24222D8046850008018DC
:10243000033820188170197800291FD11A7010BD37
:10244000104B114A6821114801F0AEF8104B114AA7
:102450006F310E4801F0A8F80F4B0E4A70210B485F
:1024600001F0A2F80D4B0B4A7121084801F09CF8CD
:10247000044B054A6821054801F096F841701A702E
:10248000DDE7C046889700107C9A0010A4970010E2
:10249000EC970010589A0010F8970010049800105C
:1024A00070B506000D001400002914D0002A14D0C5
:1024B000806873689847002806D022002900300001
:1024C000FFF79CFF280007E02A0021003000FFF7FB
:1024D00095FF200000E0100070BD0800FCE7000040
:1024E000F0B583B00500009201930AAB1C780BABEA
:1024F0001F78002C26D003685A7B944207D1012311
:10250000002B19D1002C3BD1200003B0F0BD002CD2
:102510000CD01A7B944209D81A6863001B19033B3C
:10252000D3189B78002BEBD00123E9E73E4B3F4AC1
:1025300068213F4801F038F83E4B3F4A65213F484B
:1025400001F032F803689C7B002CDBD012D01A7BA0
:1025500094420FD862001219033A19688C466244FB
:1025600051789973002900D1D97300239370537067
:102570001370C7E72C4B2D4A68212D4801F014F841
:10258000002C3AD02B681B7B9C4236D82C4BE3188E
:102590001B01AA6894466344009A1A60019A5A6023
:1025A000089A9A60099ADA602E68002C2BD030D0F5
:1025B000337B9C422DD863001B19033B3268944641
:1025C000634400229A705A701A70717B22003000A6
:1025D000FFF766FF7073844200D095E7287D009A6C
:1025E000019B00F0FFFC061E01D0002F17D00C9BB2
:1025F000002B00D188E71E7086E7124B124A3B2160
:102600000E4800F0D1FF114B114AA521084800F0F7
:10261000CBFF054B054A6821054800F0C5FF286837
:10262000210000F03FFFE2E7889700107C9A00103D
:10263000A49700101C980010889A00101C97001096
:10264000FFFFFF0F54970010109A0010189700100A
:102650006C9A0010F0B5DE4657464E464546E0B54A
:102660008BB00990002308938200B24BD6583700F4
:1026700032E0B14BB14A3F21B14800F095FFB14B78
:10268000B14A3B21B14800F08FFFB14BB14A8C21D8
:10269000AE4800F089FFB04BAE4A9021AB4800F045
:1026A00083FFA84BAD4A4021A84800F07DFF2A686F
:1026B0006B68099800F096FC00239A4698467B6860
:1026C000BFF35F8F00221A6086F310884346002B09
:1026D00051D1002800D126E100F0F8FB02000B1ECA
:1026E000C7DB00200021069007917868EFF3108681
:1026F00072B601680029FCD0BFF35F8F3968884645
:102700004C7B002C32D0BAD0097B8C42B7D894498C
:1027100065182D01B9688C46654428686968801A77
:1027200099410029C3DC01D10028C0D100214046D5
:1027300000F0AEFEA042A8D12A686B68069207930B
:10274000AB689846EB689A464346002BA3D0002C12
:10275000A7D03B681B7B9C42A3D8631EFA68D35C5E
:1027600008931B02184338610020A8E700239A460B
:1027700098460020A3E7089B1B0223439946514635
:102780001800C04705000E007A68EFF3108B72B690
:10279000136859424B41D9B2002BF9D1BFF35F8F77
:1027A000002E26DB002E52DD3B69002B53D04B451B
:1027B00072D100F08BFB02000B1E73DB01001800CE
:1027C00052197341984202D804D1914202D9012290
:1027D0005242D317002B6BDB00210491013103918E
:1027E000029451460191414600913800FFF778FE6E
:1027F00049E03B69002BD5D04B451CD1069A079B7D
:1028000010001900521BB341994202D804D19042E2
:1028100002D901225242D317002B12DB002104916E
:1028200001310391029451460191414600913800D3
:10283000FFF756FE27E04B4B464A9F21434800F0E6
:10284000B3FE3D4B3D4A3F213D4800F0ADFE002E1A
:1028500001D1002DA8D13A68002C45D0537B9C4271
:102860002CD1012100293FD1D37B002B42D1D4733D
:10287000002C52D03B681B7B9C424ED8FA68013C2E
:10288000135D0133135500233B617A68BFF35F8FFB
:1028900013608BF310881FE7324B2E4AA2212B487E
:1028A00000F082FE244B254A3F21254800F07CFEA3
:1028B000214B224A3F21224800F076FE002C0DD009
:1028C000137B9C420AD863001B19033B10688446A3
:1028D00063449B78002BC5D00121C3E7224B234AD8
:1028E0006821234800F060FE224B234AF62120484D
:1028F00000F05AFE002B0AD0117B8B4207D85900FA
:10290000CB18033B11688C4663445C70AFE7164BF1
:10291000164A6821164800F047FE0A4B0F4A40212C
:102920000A4800F041FE0BB0F0BCBB46B246A946D7
:10293000A046F0BD308C022044980010DC990010B5
:102940006098001054970010109A00101C97001007
:10295000A4980010F4990010BC980010349A00104C
:10296000FFFFFF0FC8980010889700107C9A001096
:10297000A497001004990010489A001010B50A4B53
:102980005B68002B04D00A21084800F0BFFB10BD93
:10299000054C2300064A1021206800F099FC032111
:1029A0002000FFF7B5FCEEE744040020508E022023
:1029B0008123001010B5064B5B68002B01D0044842
:1029C00010BD044B044A5C21044800F0EDFDC046F4
:1029D00044040020289900101C9A00101C97001035
:1029E000F0B5DE4657464E464546E0B58BB08046CC
:1029F00016001F00149B9A46159B994616AB1B7830
:102A00009B461F2302AA9446634400221A7032E0B8
:102A1000002809D042461268127B904204D8421E18
:102A20004146C9688A5C48E0434B444A40214448D7
:102A300000F0BAFD0798002B75D05B46002B72D0D2
:102A40004946D04704000D0003000B4300D171E05C
:102A5000002946DB00F03AFA06000F1E55DB361956
:102A60006F41B94202D804D1B04202D90126764260
:102A7000F717002F4FDB43465A68EFF3108472B606
:102A8000136859424B41D9B20791002BF8D1BFF3DB
:102A90005F8F1F3302AA9446634404930023039379
:102AA00002934B4601935346009332003B0040464D
:102AB000FFF716FD031EABD1020041464968BFF384
:102AC0005F8F00250D6084F31088002B29D01F2311
:102AD00002A98C4663441B78002BABD11202104331
:102AE000A9E732003B00361BAF41BB4202D804D1FC
:102AF000B24202D901267642F717002FBBDA114BFA
:102B0000114A3F21114800F04FFD0E4B0E4A3F2164
:102B10000E4800F049FD0B4B0B4A3F210B4800F0DB
:102B200043FD012040420BB0F0BCBB46B246A94673
:102B3000A046F0BD0798F6E754970010349A0010AD
:102B40001C97001044980010DC9900106098001049
:102B5000F8B504004268EFF3108572B61368584266
:102B60004341D8B2002BF9D1BFF35F8FCBB22268BB
:102B7000567BB3421BD10120002848D020698842EF
:102B80002BD0090AC9B2002B2ED02068007B8342CB
:102B90002AD8581EE668305C88422BD00020636833
:102BA000BFF35F8F00221A6085F31088F8BD002BF9
:102BB0000DD0167BB3420AD85E00F618033E1768A4
:102BC000BC466644B678002ED6D00120D4E7134B1D
:102BD000134A6821134800F0E7FC8521124B134A81
:102BE0004900134800F0E0FC124B134A4021104802
:102BF00000F0DAFC1900100000F054FC0028CED1DF
:102C000012210E4B094AFF31094800F0CDFC23691F
:102C10008B42C4D100232361C1E7C04688970010CE
:102C20007C9A0010A49700104C990010C4990010D1
:102C30001C97001054970010349A001070990010DF
:102C4000F0B587B006000F00FDF70DFB00281FD17F
:102C500006246442E517A4197D41BD4202D803D180
:102C6000B44201D900240025002D14DB04940595FD
:102C700000F02CF902000B1E13DBA41A9D41002D5D
:102C800017DC14D03000390000F02CF907B0F0BD8B
:102C9000234800F023FD234B234A3F21234800F023
:102CA00083FC204B204A3F21204800F07DFC002C73
:102CB000E8D0FFF77FFE0023029301931C4B0093A3
:102CC000049A059BFFF78CFE002818DADAE7002348
:102CD00000E00023002BD5D1164B1A68EFF31081CA
:102CE00072B61368002BFCD0BFF35F8F114B1B68CB
:102CF000BFF35F8F00221A6081F3108820BF049910
:102D0000059A0D4B5B6A9A42E3D80B48806A884269
:102D100003D29A42DBD00123DCE70123DAE7C04685
:102D20007499001044980010DC990010609800100D
:102D300051230010508E022000400540F8B50400D9
:102D40000D0000F0C3F802000B1E10DB200029006C
:102D5000801859418B4202D804D1824202D9012005
:102D60004042C117002908DBFFF76AFFF8BD064B98
:102D7000064A3F21064800F017FC034B034A3F2157
:102D8000034800F011FCC04644980010DC99001084
:102D90006098001010B5FA2292000023002103F081
:102DA00023F8FFF7CBFF10BD70B584B006000C0010
:102DB000FFF700FE002302930193194B00933200AA
:102DC0002300FFF70DFE051E11DD20BFFFF7F2FD0A
:102DD0002900FFF7BDFE134B5B6A9C421BD8114ACA
:102DE000926AB2421AD29C4213D0012014E00D4BD9
:102DF0005B6A9C4209D80B4A926AB24207D29C4253
:102E000001D0012008E0002006E0002004E00120BD
:102E100002E0002000E0002004B070BD0120FBE7CC
:102E2000512300100040054070B5EFF305833F20AB
:102E300018401038EFF3108C72B6194B1B68002B3A
:102E4000FBD0BFF35F8F012319008140154A516306
:102E5000154A12781400C440234214D0114B5C6A06
:102E60008300124D5B599C4206D38300104C1B59C2
:102E70008A430D490A7007E00A4A031D9B009958CE
:102E80009950002300E00023BFF35F8F044A002124
:102E900011608CF31088002B00D0984770BDC0469D
:102EA000280100D000400540A08E0220648E022040
:102EB000C085022010B50100024A0348FFF78EF9D1
:102EC00010BDC046A09A0010978E0220044B5B6A8A
:102ED000034A906A1900536A9942F9D17047C04673
:102EE00000400540084B5B6A01E0074B5B6A8B4280
:102EF000FBD301E0044B5B6A8B4203D1024B9B6A1C
:102F00008342F7D37047C0460040054070B50400C7
:102F10000D00FFF7DBFF02000B00200029008018E6
:102F200059418B4202D804D1824202D90120404249
:102F3000C117002902DBFFF7D5FF70BD024B034A22
:102F40003F21034800F030FB44980010449B0010E0
:102F50006098001070B504000D00EFF3108672B693
:102F60001B4B1B68002BFBD0BFF35F8F002D1CD0C9
:102F7000200000F057FD174B83420BD019002000B2
:102F800000F058FD0121200000F03CFD0123A3408A
:102F9000114A1360A400114BE550BFF35F8F0C4B37
:102FA00000221A6086F3108870BDA2000B4B00212E
:102FB000D1500122A2400A490B7893430B70054976
:102FC000200000F061FD0021200000F01BFDE4E77F
:102FD000280100D0292E001038600540C08502204D
:102FE000A08E0220F0B5DE4600B584B004001500C6
:102FF00001921E000293FFF769FF03958E4202D8EB
:103000004ED185424CD9EFF3108B72B6274B1B681B
:10301000002BFBD0BFF35F8F254A17780125A54011
:10302000EBB23B431370234B5D63221D9200019969
:10303000D150A2002049029850501B6A2B4212D155
:103040001C4B1B6C2B4208D00020BFF35F8F174B2B
:1030500000221A608BF3108823E0184B184AC12114
:10306000184800F0A1FAFFF731FF8E4214D802D1C0
:10307000039B834210D80E4B1B78BB420ED00D4BE6
:103080001D625D631F2004400123A3400E4A1360AC
:10309000074B1F701E38D8E70020D6E70120D4E781
:1030A000012004B080BCBB46F0BDC046280100D062
:1030B000A08E022000400540648E0220C49A0010B9
:1030C000289B0010E89A001080E200E0EFF3108CDB
:1030D00072B60B4B1B68002BFBD0BFF35F8F012335
:1030E0008340084A136208490A789A430A70BFF37A
:1030F0005F8F034B00221A608CF310887047C04624
:10310000280100D000400540A08E0220024B9C46C2
:1031100061448900016070474000003410B504002C
:10312000FFF7D8F801002000FFF7F0FFFF2323711D
:10313000BFF35F8F10BD10B50400FFF7CBF801009F
:103140002000FFF7E3FFFF23237100236371BFF328
:103150005F8F10BD034B9C46614489000160BFF343
:103160005F8F70474000003410B504000120FFF766
:10317000BFF801002000FFF7EDFF10BD10B50029DA
:103180001ED0037B99421BD84B005B18033B04689D
:10319000A4466344002919D0002A1DD0914221D0B1
:1031A000002A25D0047BA24222D80468500080184F
:1031B000033820188170197800291FD11A7010BDAA
:1031C000104B114A6821114800F0EEF9104B114ADA
:1031D0006F310E4800F0E8F90F4B0E4A70210B4892
:1031E00000F0E2F90D4B0B4A7121084800F0DCF9C0
:1031F000044B054A6821054800F0D6F941701A7061
:10320000DDE7C04688970010189D0010A4970010B5
:10321000EC970010049D0010F8970010049800101F
:1032200070B506000D001400002914D0002A14D037
:10323000806873689847002806D022002900300073
:10324000FFF79CFF280007E02A0021003000FFF76D
:1032500095FF200000E0100070BD0800FCE70000B2
:1032600010B50023437301338373037BC3730123BE
:10327000027B9A4214D9002B0CD0027B934209D8CE
:103280005A00D218033A01688C4662440133DBB21B
:103290005370EDE70B4B0C4A68210C4800F084F9A1
:1032A000002A09D0924207D8016853009A18033ABD
:1032B0008A180023537010BD024B034A682103484B
:1032C00000F072F988970010189D0010A497001064
:1032D00010B5017342608360FFF7C2FF10BD0000AC
:1032E00070B50400081E00D170BD002934D0237BC6
:1032F000994231D84B005B18033B226894466344E3
:103300005A78002AF0D02DD0237B9A422AD8530035
:103310009B18033B21688C4663445D7800215970FB
:10332000002825D0237B984222D843001B18033B5A
:1033300021688C4663440021597001002000FFF78A
:103340006FFF060029002000FFF7CAFF02003100CE
:103350002000FFF765FFC7E7084B094A68210948C5
:1033600000F022F9054B064A6821064800F01CF9D6
:10337000024B034A6821034800F016F988970010B1
:10338000189D0010A497001070B505000C001600E1
:10339000002928D02DD0037B99422AD84B005B18F6
:1033A000033B0268944663445A78002A27D19A78EE
:1033B000002A2AD11978FFF793FF0300002E03D0CB
:1033C000EA7B002A27D1EC73002B37D1002C49D09F
:1033D0002B7B9C4246D82B6861000C19033C1C19BE
:1033E0000023637070BD224B224A3821224800F02E
:1033F000DBF8224B224A6821224800F0D5F8224B04
:103400001C4A3A211C4800F0CFF8204B194A3B21B6
:10341000194800F0C9F8002A0AD0297B8A4207D847
:1034200051008A18033A29688C4662445470CAE7EE
:10343000124B134A6821134800F0B6F8002B0BD04A
:103440002A7B934208D843001B18033B2A68944602
:10345000634400229A70B9E7084B094A6821094879
:1034600000F0A2F8054B064A6821064800F09CF8D7
:10347000249C0010F09C00102C9C001088970010D9
:10348000189D0010A4970010649C00108C9C0010E4
:1034900070B504000A00457B2900FFF775FF6073D3
:1034A000280070BD70B50400002967D0437B8B42B3
:1034B0000ED0002911D0037B99420ED84B005B1827
:1034C000033B0268D0188378002B0CD1002056E013
:1034D0000121FFF7DDFF012051E0294B294A682136
:1034E000294800F061F8002B20D0227B93421DD8A0
:1034F0005A00D318033B2268D2182568EB5C8B4234
:103500001AD0002B1BD0227B934218D85A00D31814
:10351000033B2268D21853788B4216D0002BF0D18F
:103520001A4B1B4A67211B4800F03EF8144B154A02
:103530006821154800F038F84378137007E0104B05
:10354000104A6821104800F02FF843785370002388
:103550008370437001222000FFF716FF0200617B99
:10356000814205D02000FFF75BFE6073012006E07A
:10357000094B074A6D21074800F016F8002070BD7E
:1035800088970010189D0010A4970010B09C0010A0
:10359000D89C00102C9C0010B89C001000BEFDE7C9
:1035A00010B5FFF7FBFF000010B582B00C0019004A
:1035B000002A0CD0084B002A0BD001920093230064
:1035C0000200064802F0BEFE0120FFF7E7FF044BB1
:1035D000F1E7034AF1E7C046249D0010349D001036
:1035E000309D001070B52B4B2B4A1A602B4B2C4A88
:1035F0001A602C4B9A682A4B9343FAD12A4C01E06B
:1036000008CC9847294B9C42FAD300F001F9234B90
:10361000274A1A60234B9B68DB43DB01FAD1254B19
:1036200040229A675A671A67DA66234C09E0234BEF
:10363000234A83212348FFF7B7FF2000FFF76EFDE1
:103640000834214B9C4209D22368002BF5D0012B72
:10365000EDD12000FFF76FFD0834F2E71B4CA168A5
:103660001B4DC022280002F0DBFCA560FCF7FBFD2F
:10367000002800D000BEFEF71DFE00F051FBFFF752
:103680007DF9144C01E008CC9847134B9C42FAD3C7
:1036900070BDC04600E00040BFCDFBFE00F0004022
:1036A000FE7F3C0000C000403005002040050020A7
:1036B000FFFFFF0100F0014020050020649D001085
:1036C000D89D0010849D00103005002000ED00E022
:1036D0000000002040050020480500200FB400B580
:1036E00083B0084802F0FCFD049B002B07D005A91D
:1036F0000191180002F004FE034802F0F1FD0120E0
:10370000FFF74CFFC49D0010D49D0010F8B5DE46B5
:1037100057464E464546E0B505000F0092460A9AC8
:1037200093424ED31A0E91461E020A9A002330008D
:10373000494601F057FD80466C006419A4002F4BE8
:103740009C4664446368834200D260602B1FDBB2F6
:103750009B46012B3BD9C0239B01234380221201AE
:103760001A60AB00264A9958002905D0506901F02B
:10377000F7FC01300138FDD153465A0123685A4005
:10378000E0231A4080235B0123431A605A46012A32
:1037900028D980239B012343802212011A604346CB
:1037A0006360424600233000494601F01BFDAD0036
:1037B000134B58510120F0BCBB46B246A946A04667
:1037C000F8BD104B104A2D211048FFF7EDFE012FD8
:1037D000C1D1C0239B01234303221A60A368DB07E6
:1037E000FCD5C9E72168794003220A401A60A26823
:1037F0000123BB401342FAD0CBE7C0460080004013
:10380000DC860220E89D0010409E0010FC9D001008
:1038100030B583B00C2000F021FBFEF741FD0028FD
:103820000DD0002304E099002D4A2E488850013322
:10383000092BF8D92A4B2C4A5A6203B030BD2B4BC6
:1038400000229A6700F07CFB294B01221A60274B6B
:103850005B6C012BFBD1274B03221A60234B9B6B24
:10386000012BFBD1022400940533234A0121234874
:1038700000F064FA00940523214A0121214800F058
:103880005DFA214B0093002202210420FFF73EFF46
:103890001E4D00952B00002201210520FFF736FF69
:1038A000104C00942300002200210720FFF72EFF78
:1038B00000942300002200210820FFF727FF0A4B75
:1038C00000932300002200210920FFF71FFF00952D
:1038D0002B00002200210620FFF718FFADE7C046AD
:1038E000DC860220006CDC021BB700000080004078
:1038F0003CB0004030B00040002F685900800240CA
:1039000000389C1C00C00240001BB70040597307E0
:103910008000014BC0587047DC860220074B9B6833
:10392000103080001950BFF35F8FBFF35F8F044BDF
:103930000021196082F310887047C04600ED00E056
:10394000240100D010B5091A081F0A4B9C46614497
:10395000094A914208D8C30706D440104005400DDB
:10396000064B184380B210BD054B064A8B21064812
:10397000FFF71AFEFC070000FE0F000000E0FFFF4B
:10398000509E001088A00010809E001010B5091AEB
:1039900004394C08090B08D14905490D064A114361
:1039A0000180064B2343438010BD054B054A9321FC
:1039B0000548FFF7F9FDC04600F0FFFF00F8FFFFE4
:1039C000BC9E00105CA00010809E0010012383406C
:1039D000034A10681840431E9841C0B27047C04661
:1039E00000E100E0002904D0034B1860034B18608D
:1039F0007047034B1860FBE780E200E000E100E065
:103A000080E100E010B5012383401800FFF7EAFFD2
:103A100010BD000001238340014A13607047C04677
:103A200000E200E0024B9B6810308000C0587047F5
:103A300000ED00E070B504000D00EFF3108672B6E3
:103A40000C4B1B68002BFBD0BFF35F8F2000FFF7F0
:103A5000E9FF094B984201D0A84205D13200290064
:103A60002000FFF75BFF70BD044B054A6E2105483F
:103A7000FFF79AFD240100D0CD010010CC9E00106C
:103A8000A4A00010809E0010F0B5CE46474680B539
:103A900083B006000D00EFF3108872B6564B1B681A
:103AA000002BFBD0BFF35F8F544B9A683400103467
:103AB000A300D758524B9F4207D0AF4200D199E0A4
:103AC0000197504BFB1A2F2B09D942463900300081
:103AD000FFF724FF03B0C0BCB946B046F0BD3000CC
:103AE000FFF774FF814600213000FFF78BFFBFF323
:103AF0005F8FFCF7B8FB002801D0844211D101236D
:103B0000019C9C430022A368AB4212D00622A2561D
:103B1000002A0DDB53009B189B002200394CE4184F
:103B2000F1E71E21384B394AFF313948FFF73CFD98
:103B30002200AB4257D106256557002D39DB6B00BB
:103B40005B199A002F4B9B189A68A260DA79E27190
:103B500006229A56A2719B795BB2002B10DABD2027
:103B60000002A0806B005B199B00264AD318294AEB
:103B700011789971157049463000FFF743FFA4E7AB
:103B8000201D6B005B199B001E4A9B181A1D9B8809
:103B9000D90A1C2907D15B055B150233590051185E
:103BA000FFF7D0FEDDE71C4B1C4A99211848FFF7B0
:103BB000FBFC002812D1002A0ED0FF239371184B72
:103BC0009380144A1378A371164B0E49641A64410A
:103BD00063431B0D1370CEE7094FF2E7201D124916
:103BE000FFF7D4FEC7E75221104B084AFF310848BF
:103BF000FFF7DAFC024F68E7240100D000ED00E097
:103C0000CD0100106C040020E09F001074A0001093
:103C1000809E0010998E0220C89F001094A0001072
:103C200000BDFFFFAAAA0000A604002004A0001007
:103C300070B50400012606432D4BF31A2F2B28D80C
:103C4000FCF711FB00282BD0EFF3108C72B6294B38
:103C50001B68002BFBD0BFF35F8F274D2200244948
:103C6000521A524155432D0D6DB2244B9B68800072
:103C70001B58B3421BD00022032A32D853009B1892
:103C80009B001B49CB189B795BB2AB421FD0013222
:103C9000F2E7BB211A4B1B4A49001B48FFF784FC83
:103CA0007A211A4B174AFF311748FFF77DFC134B57
:103CB0009B68174A1A50174B1A78A2711D70BFF3F0
:103CC0005F8F0C4B00221A608CF3108870BD0800C7
:103CD0005300991889004118FF268E710E4A8A8078
:103CE000E9E7C5210D4B074A49000748FFF75CFC8F
:103CF0006C040020240100D0AAAA000000ED00E01E
:103D00000CA0001040A00010809E001034A00010F5
:103D1000CD010010998E022000BDFFFFB09C001065
:103D20000022044B02E0044902C30132072AFAD9F7
:103D30007047C04600E400E080808080F0B5CE4649
:103D400000B504000F0091461D000C2001F008FA98
:103D5000060043011B1A9901C91AC90009188901F3
:103D6000484601F0FDF90200103A98235B009A42A0
:103D700033D86B1E062B36D8069B013B062B32D858
:103D8000069B9D4235D34B461A09B24237D32D04C8
:103D9000069B1E0335432368002B36DB254B9C42D4
:103DA00044D080225201244B1A60244B1A60244BC9
:103DB0009B6811009943FAD12760A060231DC0229F
:103DC00092011A43212313602368002BFCDAE5607B
:103DD0000823136080BCB946F0BD1A4B1A4A16215D
:103DE0001A48FFF7E1FB1A4B174A19211748FFF74A
:103DF000DBFB184B144A1F211448FFF7D5FB164B69
:103E0000114A22211148FFF7CFFB22683F231340BC
:103E1000BB42C3D1A3681B051B0D8342BED1E3681F
:103E2000EE22D2021340AB42B8D1D3E780229201F6
:103E3000B9E7C04600C0024000E0004000F000408A
:103E400000C00040C0A0001098A10010DCA000102D
:103E500018A1001064A100107CA1001080239B0019
:103E60000343014AD362704700800540024B1A6841
:103E7000024B5A607047C046A88B02200080054064
:103E800010B50200164B8020C0051860154B16486F
:103E9000186000290AD0154BE021C9041960002AD6
:103EA00009D1124B802212061A6010BD0C4BE02182
:103EB000C9041960F3E753019B1A980080180001A8
:103EC0000B4B186080235B04984202D3084B094ACD
:103ED0001A60FFF7CBFF054B8022D2051A60E4E79A
:103EE00000B0054008200140FCFF010000A0054093
:103EF000A88B0220FFFFFF0010B5030010000C4A42
:103F00008024E4051460002B0DD001221343094ADC
:103F1000094CD461094C5C401462516293620021E7
:103F2000FFF7AEFF10BD034B0022DA61F7E7C04692
:103F300000B0054000800540D3C007B02D3FF84FCA
:103F4000064BAA2212011A602F22DA60044B054A9E
:103F50001A60024B5B68002BFBDA7047004002409E
:103F60000060024000B0FA00704710B5002802D08F
:103F70000B684968984710BD0100002007E08300E6
:103F80001B185B00501C08601078C01830380A6895
:103F90001378303BDBB2092BF1D97047F0B5DE4620
:103FA00057464E464546E0B583B093461F000C9BEE
:103FB0009A460D9C0E9B99460F9B9B0703D0B846D3
:103FC0000F00060022E00192A34688464E46B946FD
:103FD0000700B44207D2551C4B4641462020B84743
:103FE00001342A00F5E73D004F465C46019B9B46A5
:103FF000B1464646B84637002E0007E0013C551C46
:104000005346185D43463900B0472A00002CF5D1CD
:1040100035003E0047460F9B9B0707D4100003B0B6
:10402000F0BCBB46B246A946A046F0BDB0464E46DF
:10403000B9462F005D46531BB342EFD2541C4B468A
:1040400041462020B8472200F5E7F0B5CE46474666
:1040500080B585B0944698460C9D0D9C0EAB1B78A0
:104060009946109A119B129EB7071CD4002B0CD0B6
:10407000F7070AD54F46002F02D10C37374204D03C
:10408000013B02E030272F550134944201D21F2C0E
:10409000F8D9F70707D59C4205D21F2C03D8302743
:1040A0002F550134F5E7F70615D5770505D4002C13
:1040B00003D0944224D09C4222D00F9A102A2BD0B5
:1040C0000F9A102A30D00F9A022A35D01F2C02D80E
:1040D00030222A5501341F2C05D84A46002A31D0F7
:1040E0002D222A55013403960293019400954346EC
:1040F0006246FFF753FF05B0C0BCB946B046F0BDFD
:10410000621E012C06D00F9F102F01D01400D4E79F
:10411000023CD2E71400D0E7B206D1D41F2CCFD88E
:1041200078222A550134D1E7B206CCD51F2CCAD843
:1041300058222A550134C9E71F2CC7D860322A55A6
:104140000134C3E7720703D52B222A550134CAE78D
:104150003207C8D520222A550134C4E7F0B5DE461F
:1041600057464E464546E0B593B081468A4608928A
:1041700009931CAB10CB1B789B461E9D219B984638
:10418000002C03D1102342469A4390468023DB0043
:1041900046461E4042461A4212D0002C22D000262B
:1041A0000EE03033D9B2771C0AAB995529002000B4
:1041B00000F0D6FFAC4216D31F2F14D83E000400E7
:1041C0002900200000F0CCFFCBB2092BE9D94246F0
:1041D000920605D54121C918C9B20A39C9B2E2E728
:1041E0006121F8E7270043460693209B05931F9B18
:1041F000049303955B46029301970AAB0093099BD6
:10420000089A51464846FFF720FF13B0F0BCBB4662
:10421000B246A946A046F0BDF0B5DE4657464E462A
:104220004546E0B595B0089009910A920B931E9E01
:104230001F9C20AB1B789B46229B9946239D269B67
:104240009A463300234303D1103352469A43924691
:104250008023DB0057461F4052461A4219D03300D4
:1042600023432DD0002714E03033DAB27B1C98466C
:104270000CABDA554A462B003000210000F0B2FFAB
:10428000A5421FD819D043461F2B1BD8474606000E
:104290000C004A462B003000210000F0A3FFD3B2EF
:1042A000092BE1D95246920605D54122D218D2B245
:1042B0000A3AD2B2DAE76122F8E7B145E3D901E080
:1042C0000023984653460693259B0593249B04930D
:1042D0004B4603935B460293434601930CAB00931A
:1042E0000B9B0A9A09990898FFF7AFFE15B0F0BC2E
:1042F000BB46B246A946A046F0BD0000F0B5DE467A
:1043000057464E464546E0B591B083468A460C92E4
:1043100098461A9C08941B9D099522002B002000AA
:10432000290001F0EEF9002800D0E5E00122524218
:10433000D74B2000290001F0DFF9002800D0DBE096
:1043400001225242D34B2000290001F0BFF900287E
:1043500000D0D1E000220023089E3000099D2900F2
:1043600001F0B4F9002800D0DDE008980999069022
:1043700007918023DB001E9A1A400D921E9A1A4262
:1043800001D106231C930698079904000D000A002A
:104390000600024300D1D1E0080D4005400DBE4C9F
:1043A000A44660440A03120BBC4B13431F0001F0E8
:1043B000BBF9BB4ABB4B01F046F9BB4ABB4B01F012
:1043C0001BF904000D000022B94B3000390001F048
:1043D0000AF9B84AB84B01F036F902000B00200088
:1043E000290001F009F901F0B7F9814601F09CF9C3
:1043F00004000D00B14AB24B01F025F90022B14B87
:1044000001F0FAF801F0A8F90600AF4AAF4B20001E
:10441000290001F018F904000D00300001F084F9C2
:10442000AB4AAC4B01F00FF902000B002000290051
:1044300001F0D9F804000D0002000B0001F003F9AF
:104440000A900B91A44BF31800261F0522002B00A5
:104450002000290001F0D0F80E900F9122002B00CF
:1044600000208021C90501F0BEF804000D000022E3
:104470009A4B0A980B9901F0C8F80022984B01F06A
:10448000BBF802000B000A980B9901F0BEF800225D
:10449000944B01F0B1F802000B000A980B9901F05F
:1044A000B4F802000B002000290001F0A5F802007A
:1044B0000B000E980F9901F0A8F80022774B01F03D
:1044C0009BF832003B0001F0BEF806000F0004002C
:1044D0000D00069A079B01F00FF9002830D0012348
:1044E0005B429C46E14400227D4B3000390001F0E4
:1044F0008CF804000D0023E01E9B04931D9B039386
:104500001C9B0293089A099B0092019343460C9AC4
:104510005146584600F0FCF811B0F0BCBB46B2461C
:10452000A946A046F0BD00230024069307940696F2
:1045300080231B069C46654407951AE7002399468D
:104540004B466333C62B1ED804261E9B1B0526D55F
:104550002B0023430FD0644A644B0698079901F05F
:10456000C3F8002879D00022614B0698079901F022
:10457000ADF8002871D01C9B4B4506DD4A46981AC1
:10458000431E1C9303E00526DFE700231C938023D2
:10459000DB001E9A1A431E920026002399461D9B9B
:1045A0009E4264D29F1B02231E9A1A400A921E9AB0
:1045B000134202D0002E00D000274B46002B07D01C
:1045C00022002B000698079901F01FF8069007912A
:1045D000002200230898099901F078F8002848D1B2
:1045E000444B1E9A1340049303971C9B0293069B13
:1045F000079C0093019443460C9A5146584600F09C
:1046000087F8002E00D187E71E9B9B063DD54525E8
:10461000441C4346020051462800D8474B46DA174F
:104620009B18534005220592013E049600220392F6
:104630000A3202924A46D00F01900093434622006C
:1046400051465846FFF78AFD0A9B002B00D163E7CD
:1046500002005F460C9E1D9D54E01C9B002B9ED0CB
:104660000D9B002B9BD01C9B013B1C9397E70027C5
:1046700099E7069C079D22002900802000068446B9
:1046800061440B0006920793AAE76525C0E7C04680
:10469000FFFFEF7FFFFFEFFF01FCFFFF0000F03F98
:1046A000FB799F501344D33FB3C8608B288AC63F21
:1046B0000000F83F61436F63A787D23F71A3790978
:1046C0004F930A400000E03F1655B5BBB16B024066
:1046D000EF39FAFE422EE63FFF03000000002C40B7
:1046E00000002440000018402D431CEBE2361A3F26
:1046F00080842E41FFF7FFFF541C43465146202083
:10470000B8472200931BAB42F6D3100004E7C04623
:10471000F0B5DE4657464E464546E0B595B00690A4
:10472000079193469946209F1E9A1F9B10001900DF
:1047300000F0E7FF002831D101225242BF4B1E9802
:104740001F9900F0C3FF002837D101225242BC4B11
:104750001E981F9900F0D0FF00283DD10022B94BD0
:104760001E981F9900F0C8FF002850D10022B64BB8
:104770001E981F9900F0AAFF002848D100220023AC
:104780001E981F9900F0A2FF002850D100239846E0
:10479000229B5B0500D4B6E0002458E0229B0393E3
:1047A000219B029303230193A84B00934B465A4647
:1047B00007990698FFF7F2FB0EE1229B0393219BDA
:1047C000029304230193A24B00934B465A46079948
:1047D0000698FFF7E3FBFFE00423229A1A40229990
:1047E0000B4210D09B4B002A0FD004222299039138
:1047F00021990291019200934B465A4607990698D7
:10480000FFF7CCFBE8E0944BEDE70322EEE7229BB9
:104810000493219B039302971E9B1F9C009301947A
:104820004B465A4607990698FFF768FDD4E01E9A52
:104830001F9B0020002100F0D6FE1E901F91012337
:104840009846A5E70CAB30221A55013F01341F2CC6
:1048500001D8092FF6D81E981F9900F07DFF05009A
:1048600000F062FF02000B001E981F9900F0BBFED3
:10487000FA007A4B9B181A685B680A920B9300F057
:10488000E2FE0890099100F08BFF060000F048FF5F
:1048900002000B000898099900F0A5FE0890099104
:1048A00000226F4B00F028FF00282ED00136300088
:1048B00000F036FF02000B000A980B9900F00CFF85
:1048C000002801D001350026002F2CD1280000F04F
:1048D0002BFF02000B001E981F9900F084FE0600BB
:1048E0000F0000225E4B00F0F1FE002846D10022AE
:1048F0005B4B3000390000F0FFFE00283ED1EB0793
:104900003CD501353AE0062746E70022544B08988B
:10491000099900F0DBFE0028D6D1002E01D0F30764
:10492000D2D50136D0E7AA461F2C11D8013F0A2163
:10493000300000F015FC651C30310CAB19550A2114
:10494000300000F00DFC092E0ED906002C00EBE71C
:1049500055461F2C0CD87B1E002F09D00CAA3021E5
:1049600011551F000134F4E72B0055461C00F0E7F9
:104970001F2C03D80CAB2E221A5501341F2C10D833
:104980000A21280000F0C4FB661C30310CAB19551D
:104990000A21280000F0BCFB051E01D03400EDE721
:1049A00034000323229A1340012B1CD01F2C06D85D
:1049B0004346002B32D00CAB2D221A550134229BDA
:1049C0000393219B029301940CAB00934B465A46F0
:1049D00007990698FFF7E2FA15B0F0BCBB46B2465D
:1049E000A946A046F0BD219B002B13D04346002BC7
:1049F00002D10C3313420FD0219B013B21931900AC
:104A000003E00CAB30221A5501348C42CED21F2C5D
:104A1000F7D9CBE72199F8E72199F6E7229B5B07C5
:104A200004D50CAB2B221A550134C8E7229B1B0777
:104A3000C5D50CAB20221A550134C0E7FFFFEFFFAC
:104A4000FFFFEF7F65CDCD4165CDCDC1B0A1001099
:104A5000B4A10010A8A10010A4A10010A0A30010F0
:104A60000000E03FF0B5DE4657464E464546E0B50D
:104A700093B082468B4690461193002900D1EBE219
:104A800000275546119B1878002800D1E7E2252819
:104A900009D07C1C43463A005946A847119B013374
:104AA00011932700EEE7013311930024119A117836
:104AB0000B00203BD8B2102803D88300D048C3583D
:104AC0009F460B00303BDBB2092B2CD92A292FD073
:104AD00000230A93119B1A782E2A39D000239A4674
:104AE000119A1378683BD9B2122976D88B00C54940
:104AF000CB589F4601231C4301321192D6E7022373
:104B00001C4301321192D1E704231C43013211925C
:104B1000CCE708231C4301321192C7E710231C4342
:104B200001321192C2E711A8FFF726FA0A90D1E7E5
:104B30001C9B1A1D1C921868002804DB0A90119B0C
:104B400001331193C6E702231C4343420A93F6E75D
:104B50008022D20014435A1C11925A781300303B21
:104B6000DBB2092B04D92A2A07D000239A46B7E7DB
:104B700011A8FFF701FA8246B2E71C9B1A1D1C928E
:104B80001868002804DB8246119B01331193A7E7C4
:104B90000020F8E780235B002343511C11915278D9
:104BA0006C2A01D01C0018E0C0239B001C4301317B
:104BB000119112E080232343511C11915278682AED
:104BC00001D01C0009E0C0231C430131119104E015
:104BD00080235B001C4301321192119B1878030063
:104BE000253BDAB2532A00D92CE29300864AD358E7
:104BF0009F4680239B001C4301321192EDE78023E6
:104C00005B001C4301321192E7E7782809D058284D
:104C100038D06F2838D0622838D010239C430A2619
:104C200000E01026582833D0692803D0642801D02A
:104C30000C229443630501D50122944369282AD0AC
:104C4000642828D0A30500D59FE0E30500D5B8E08F
:104C5000630600D4CAE01C9A111D1C911168FF2242
:104C60000A4005940A9B049353460393029600233B
:104C70000193009243463A0059462800FFF76EFA26
:104C8000070027E01026CDE70826CBE70226C9E774
:104C900020221443C8E7A30520D4E30550D46306BB
:104CA00066D51C9A111D1C911168FF220A40D3176A
:104CB000D118594005940A9B0493534603930296D6
:104CC000D20F0192009143463A0059462800FFF75F
:104CD00045FA0700119B01331193D3E61C9BDA1DA3
:104CE00007218A43110008311C91116853689C46C2
:104CF000DB170C930D930C9A0D9B100048400E90FF
:104D0000624653400F930E980F990C9A0D9B801A90
:104D100099410E900F9108940A9B0793534606936E
:104D20000496002305936346DA0F029200900191E6
:104D300043463A0059462800FFF76EFA0700C9E7D4
:104D40001C9A111D1C911268D317D1185940059453
:104D50000A9B0493534603930296D20F019200914B
:104D600043463A0059462800FFF7F8F90700B1E733
:104D7000230605D51C9A111D1C910023D25E96E7CF
:104D80001C9A111D1C91126891E71C9BDA1D0721CA
:104D90008A43110008311C9108940A9B07935346DB
:104DA00006930496002305930293136854680093B6
:104DB000019443463A0059462800FFF72DFA0700B0
:104DC00088E71C9A111D1C9105940A9B0493534675
:104DD00003930296002301931368009343463A001D
:104DE00059462800FFF7BAF9070073E723060DD5E7
:104DF0001C9A111D1C9112681204120C31E7C04656
:104E0000BCA1001000A200104CA200101C9A111DA1
:104E10001C91126825E746281AD01C9B07330722ED
:104E200093431A0008321C9204940A9A0392524641
:104E300002925C681B680093019443463A0059460D
:104E40002800FFF765FC0700119B0133119319E659
:104E500020231C43E1E7672801D0472802D18023A3
:104E60001B011C43452801D0472801D120231C43A6
:104E70001C9B0733072293431A0008321C920494A8
:104E80000A9A0392524602925C681B68009301944E
:104E900043463A0059462800FFF730FA0700119BB5
:104EA00001331193EEE502231A0022409246234279
:104EB0001FD001241C9B1A1D1C927A1C9146187845
:104EC00043463A005946A8475346002B16D1119B3A
:104ED000013311934F46D5E5561C434659462020D1
:104EE000B847230032005C1C9D42F5D83D001700F6
:104EF000E0E701233A002F000A9DF4E74A46A9465D
:104F00000A9D06E0571C434659462020C8473400F6
:104F10003A00661CA542F5D84D469146D7E71C9B42
:104F20001A1D1C921B6899465346002B00D1013B69
:104F30004E4601E0013613003278002A02D05A1E94
:104F4000002BF7D14B46F21A10928023DB0026008B
:104F50001E401C4203D0524501D9534610930223F0
:104F60001A0022400B92234205D03A0037004C46EB
:104F7000A946554620E03A00109B5F46B3462E00F6
:104F800006E0551C434639002020B04723002A0084
:104F90005C1C0A999942F4D835005E46BB461094D1
:104FA00037004C46A946554606E01D000134561C04
:104FB00043465946C84732002078002804D0002FC5
:104FC000F4D06B1E002DF0D117004D460B9B002B2B
:104FD00003D1119B0133119354E50A9F109B06E006
:104FE000561C434659462020A847230032005C1C2B
:104FF0009F42F5D81700ECE721231C431C9B1A1D88
:105000001C921B6800930594082304935346039352
:10501000102302930023019343463A005946280087
:10502000FFF79CF80700119B013311932AE57C1CC4
:1050300043463A0059462520A847119B0133119356
:1050400027001FE57C1C43463A005946A847119BA0
:1050500001331193270015E50A4B9A4610E5AA463D
:10506000474502D343465A1E00E03A00434659469C
:105070000020D047380013B0F0BCBB46B246A9466A
:10508000A046F0BD693F001000B585B002900391C5
:105090000121009313004A4202A90248FFF7E2FCF3
:1050A00005B000BD6B3F001001480421014B1847BB
:1050B000C0040020D950001010B5010018231B882F
:1050C00014221088984710BD10B5010018231B88C2
:1050D00016221088984710BDF0B5C64600B50700E7
:1050E0000E0000250123984600E00135B5420AD2A2
:1050F000AC003C192068FFF7DFFF20600028F4D1E6
:1051000000239846F1E7404680BCB846F0BD000059
:10511000124A936F9B0815D29066D166002905D07C
:10512000FFE7FFE7FFE7516F106F704704B580217D
:105130000906C2175140002800D0C84304F09CF96A
:10514000002104BDF0B5146E556E576F166FFFF752
:10515000E3FF1466556657671667F0BD000000D080
:10516000114A936F9B0813D210665166002905D02F
:10517000FFE7FFE7FFE7516F106F704704B50028A6
:1051800001D00020C04304F077F9002104BDC046DF
:10519000F0B5146E556E576F166FFFF7E5FF146686
:1051A000556657671667F0BD000000D094464E4A1A
:1051B000926F9208624601D230E0C046F0B54A4E86
:1051C000B56F6D08FCD3346E756E776F366F00F077
:1051D00025F89446444A1466556657671667624632
:1051E000F0BDC0469446404A926F9208624601D292
:1051F00058E0C046F0B53C4EB56F6D08FCD3346E38
:10520000756E776F366F00F04DF89446364A146627
:105210005566576716676246F0BDC046002B24DB13
:1052200011D000293EDA00B5C943404200D1013116
:1052300000F038F8C943404200D10131DB4352420B
:1052400000D1013300BD002AEBD1002801D1002993
:1052500005D00020C90FC90701D1C043410800B5DE
:1052600004F002F90022002300BD00B500290ADB8A
:10527000DB43524200D1013300F014F8C9434042ED
:1052800000D1013100BDC943404200D10131DB43AF
:10529000524200D1013300F005F8DB43524200D105
:1052A000013300BD002923D1002B18D1002A0CD0D6
:1052B000BC460D4F38667A6600210023FFE7FFE702
:1052C000FFE77A6F386F67467047002801D00748BC
:1052D000010000B504F0C8F80022002300BD020060
:1052E0000B00002000217047000000D0FFFFFFFFEF
:1052F000002B00D0BFE0130C28D1002AE7D080B4E7
:10530000114F39667A66FFE7FFE730B4040C7B6F14
:10531000396F1B0423433B667A66FFE7FFE7FFE72D
:10532000C04684B27B6F3D6F1B0423433B667A66A5
:10533000FFE7FFE7C04600232C042D0C7A6F386F7F
:1053400000196941B0BC7047000000D0F0B5944628
:105350000025140E01D112020835140F01D11201DB
:105360000435940F01D192000235D40F01D15200BF
:105370000135D40B0134254F7C66254C3C660E0C60
:1053800093B2FFE7FFE7FFE73C6F6643360C770316
:10539000BE467343DF0B5B04C01AB941130C734361
:1053A000DB18C91ACE086643360CB64493B2734371
:1053B0001F0F1B01C01AB941130C73431F0B1B05B0
:1053C000C01AB941860D8F023E436643360C092D43
:1053D00024DB520A7243801A7703460A6643360C6E
:1053E00016235B1BDE40DF40BF1964466643821B09
:1053F0007046043506330100D940A840C01900D3D7
:105400000131A24206D20023F0BD0000000000D00E
:10541000FFFFFFFF121B0130F3D3F1E709277F1BCA
:10542000FE406446A2B27243801A00D20139220CB7
:105430007243130C1204821A99410B007046043512
:1054400013370100F940A840801900D30131002B27
:1054500002D1A2420AD2F0BD013000D30131121BA9
:10546000FAD2013BF8D1A24200D2F0BD013000D304
:105470000131121BF7E7F0B51C0C00D080E00CB432
:1054800000251C0A04D11B02160E334312020835F4
:105490001C0B04D11B01160F3343120104359C0B66
:1054A00004D19B00960F334392000235DC0B02D1EE
:1054B00092185B4101351C00971864410134464F36
:1054C0007C66464C3C660E0CFFE7FFE7FFE7C046F4
:1054D0003C6F6643360C7703BE4697B27743C01BDA
:1054E00000D20139C01B00D201399FB27743C91BDA
:1054F000C91B170C77437E04FF0B801BB941CE08F4
:105500006643360C0C2D33DBB644120B1F053A43B1
:105510001B0B97B27743C01B00D201399FB2774370
:10552000C91B170C77433E043F0C801BB941860D05
:105530008F023E43664329277F1BFE400C3D774682
:10554000AF40BF1930BCA2B2ABB272437343801AF2
:105550009941220C7243130C1204801A99410200E3
:105560000B000137001BA941F9D2781E0021F0BDC4
:105570000C277F1BFE4077467F0BAF40FF19E0E70B
:1055800000245D1C07D0144F7D663966FFE7FFE7F6
:10559000FFE7FFE73C6F95B29EB265436643401B51
:1055A000B141150C1E0C6543664336042F0C3E4377
:1055B0002D04401BB141994204D202000B0020008F
:1055C0000021F0BD01D19042F7D3801A99410134F6
:1055D0009942F2D3F6E70000000000D0FFFFFFFF82
:1055E00048404140484018B41B4B5B68FC4601935F
:1055F00008BD04DFBB58001018B4174B1B68FC46ED
:10560000019308BD00DFC55800109446134A926FFD
:10561000920809D2624618B40F4BDB68FC4601932E
:1056200008BD0CDF7D5B00100C4AF0B5146E556EA2
:10563000576F166F6246FFF7EEFF084A146655660D
:1056400057671667F0BD18B4034B9B68FC4601937F
:1056500008BD08DF215A00104C8C0220000000D049
:10566000FFB550404240504059404B40594000E047
:10567000FFB5154F4C00640D03D0BC4204D10C03A0
:1056800014D80020090D09055C00640D03D0BC424C
:1056900004D11C030AD800221B0D1B0501264B4018
:1056A00009D44B4003D58B4200D18242FFBD9942C1
:1056B000FCD19042FFBD0B43DB1803431343F5D0ED
:1056C000C9434918FFBD0000FF07000000B5FFF700
:1056D000CFFF804100BDC04600B5FFF7C9FF01D92B
:1056E000002000BD012000BD00B5FFF7B9FF01D9C2
:1056F000002000BD012000BD00B5FFF7B1FF8041D3
:1057000000BD012040054A00121804D85A001218A2
:1057100001D800207047012070470020704700002A
:105720000021002805D17047C1174840401AFAD01F
:10573000C90713B5064B1B6898470CBC441CA24014
:105740001005120B0349091B09051943114310BD2C
:105750004C8D02201F04000010B54C00620D802308
:10576000D218DB00D21A5B057E2A10DD9E3A13DACE
:10577000CC170903490819435242D140640001344F
:105780001532202A05DAD0400843604310BD0020BE
:1057900010BD0846604310BDC80FC018013810BDC9
:1057A00018B4044B5B6AFC46019308BD24DF2D5DF1
:1057B000001000004C8C022070B513231C78012CC3
:1057C00014D0012C14DC022C02DC1F4A1F4B9A64FB
:1057D0001F48FFF771FC1F4B186070BD99001A48F5
:1057E0001A4A885001331F2BF8D9EAE70023FAE759
:1057F0001948FFF769FC05001848FFF765FC0238F7
:1058000003789B007F2B19DD802229000F4800F0D0
:1058100007FC022CD7D1124B1A88B5231B029A42DF
:1058200009D1104B1A88104B9A4204D10F4B1A8899
:105830000F4B9A42C7D00020FDF750FF0D4B0E4A88
:1058400032210E48FDF7B0FE815800104C8C02202A
:105850004C3300004C8D022053440000534600009E
:1058600054380000D8380000494600009C38000039
:1058700059460000F0A3001098A4001050A4001096
:1058800007B56046002800D100BE01880A0A023030
:10589000DF2AFAD1C9B2820804D302884088000402
:1058A000104300E00068024A5050039007BD00001A
:1058B0004C8C02200FB403BC0CBCF0B50124E407EF
:1058C000634000E0F0B50C0DCF0F661E3605891B56
:1058D000640503D3C943404200D30131640D03D0B2
:1058E000661CF60A07D0E41B00207F00791C89079C
:1058F0008912803C24031D0DDF0F6E1E36059B1B95
:105900006D0503D3DB43524200D301336D0D03D049
:105910006E1CF60A07D0ED1B00227F007B1C9B0744
:105920009B12803D2D032F1B661B58D4A446202EAE
:1059300046DA20371400BC401D00BD40F240334120
:105940002A4380185941CB0F05D0C943C0430022D8
:1059500064425041514162464D0D28D10D0D07D191
:1059600000281FD0241940414941013A0D0DF9D0BA
:10597000640006D3013000D30131002C01D140086E
:105980004000013A0BD4941CE40A04D112051144DE
:10599000DB071944F0BDD907204B194300E0D907B4
:1059A0000020F0BD0029DDD1002CDBD1F0BD01329B
:1059B000C6074008CD0728434908002EE1D0D9E7A3
:1059C0003C2E29DA203E40371400BC4000D0012490
:1059D000F24014431A00BB401C43D317ACE7AC465B
:1059E000202F08DA20360400B4400D00B540F840FE
:1059F00039412843A5E73C2F0CDA203F403604000C
:105A0000B44000D00124F84004430800B1400C43E6
:105A1000C117EAE710001900002494E70000F07FA6
:105A2000F0B50C0D661E3605891BE60A6405640D8B
:105A300002D0651CED0A04D0002001210905803C3C
:105A40002403A4461C0D671E3F05DB1BE70A640503
:105A5000640D02D0651CED0A04D0002201231B0551
:105A6000803C24037740644497B484B296B2744374
:105A7000070C7E43150C6F4380B26843361802D37F
:105A8000012000043F183004350C00197D41844684
:105A900088B29AB250430C0C62431F0C7C438EB206
:105AA0007E43921902D301263604A4191604170C5A
:105AB0003618674101BC81B29AB25143040C62436B
:105AC0001B0C5C4380B25843121802D3012000041F
:105AD00024181004130C401863412D185E41002057
:105AE000474106BC88B293B258430C0C6343120C76
:105AF000544389B251435B1802D30121090464184D
:105B000019041A0C091862416D18564100204741CA
:105B100018BCF902720D1143F0026A0D1043ED0238
:105B20000A0D03D16D1940414941013B124E9B1BA7
:105B30007600B3420ED26D0007D3013000267141CA
:105B40006646354301D1400840001B05C918E407EB
:105B50002144F0BD0BDA013306D1013004D101310B
:105B60004F0D01D04908F2E7E1070020F0BD0136F2
:105B700031050020EBE70000FF030000F0B51C0D2D
:105B8000671E3F05DB1BE70A6405640D02D0661C37
:105B9000F60A04D0002201231B05803C2403D025F3
:105BA0002D060026F6432E661E096E66CE0FF619E8
:105BB000B44649004F0D02D07E1CF60A03D00020E7
:105BC0000021403F3F033E1BB600B444013F7F0528
:105BD000C91B49082E6F013676089C02950D254396
:105BE0007543ED137543AD1301356D10F603761B48
:105BF0000CB4CC02450D2C43A2B2B3B25A43270CCD
:105C00007B43350C6F43A4B26C431B1902D30124B0
:105C100024043F191C041D0CA4187D4124196D4156
:105C2000009A91B2ACB26143170C7C432B0C5F43DA
:105C300092B25A43A41802D301221204BF182204BC
:105C4000230C52187B41019C6C431B19520ED90145
:105C50000A434401A01A81B2B2B2514303145A4319
:105C6000360C734387B27743D617D21900277E418B
:105C700036049B191704160C7F185E417316ED1835
:105C8000F301002680337541A90F06D16400690A2B
:105C9000E8055B0A184309D22FE0042294448033BC
:105CA0007541A90AA8059B0A184326D340414941DA
:105CB0002404009A019B0D005543641B4343E41ADE
:105CC00095B286B27543170C7E43030C5F4392B2C4
:105CD0005A43B61802D301221204BF183204330CFF
:105CE00052197B4152429C41002C02D400220130C7
:105CF00051414008CA071043490802B06246D7071D
:105D00009210084BD218084B9A4203D212058918F8
:105D1000C919F0BD0020002A01DC3900F0BD0133B3
:105D20001905F5E7FD030000FE070000002200B59D
:105D3000203200F004F8080000BD000000220B151E
:105D40000AD410B5944600F031F81414013400DA86
:105D50000021CB17144C20470020002170476244DB
:105D6000343A0CD40C2A07DA040091409040524295
:105D70002032D440214310BDD843D94310BD203236
:105D800007D40C469440524220321141D040204367
:105D900010BD0800C917203203D4524220321041EE
:105DA00010BD1800190010BD5F5D00100A0DCC0F6A
:105DB000531E1B05C91A520503D3C943404200D3E1
:105DC0000131520D03D0531CDB0A07D0121B0020F7
:105DD0006400611C89078912803A1203014BD21AB0
:105DE00070470000FF03000051434343C9188C462D
:105DF000110C83B24B4310B4040C614392B280B2D5
:105E0000504362431C041B0C001910BC594113047D
:105E1000120CC01851416144704700004840414095
:105E2000484000239C46114B5B68184700239C4662
:105E30000E4B1B6818470E4A936F9B0804D2002331
:105E40009C460A4BDB681847F0B5146E556E576FC9
:105E5000166FFFF7F4FF064A146655665767166714
:105E6000F0BD00239C46014B9B681847508D0220D3
:105E7000000000D0491A002808D1084670470000E9
:105E8000C10FC90700D54042002817D0F44603B41B
:105E90000B4B1B68984706BC81409E3840428031BE
:105EA00007D20B0607D04900490AC0051043084332
:105EB00060470130F8E7490A8902F5E770470000BA
:105EC0004C8D022000239C46014B5B6A1847000062
:105ED000508D022070B513231D782A48FFF7F4F87F
:105EE0000400012D11D0012D09DDA31E1B789B009C
:105EF0007F2B40DD80222100234800F091F82348C9
:105F0000FFF7DAF8224B186070BD542201001E48DA
:105F100000F086F81F4B1A881F4B9A421CD1A7230A
:105F20009B011A881D4B9A4216D11D4B1A881D4B96
:105F30009A4211D11C4B1A8894239B019A420BD18F
:105F40001A4B1A881A4B9A4206D11A4B1A681A4BE6
:105F50009A4201D1152307E01848FDF7BFFB9900CD
:105F60001748094A885001331F2BF8D9144A064BA9
:105F70001A62DA61B7E7134B134A42211348FDF75F
:105F800013FBC04653460000508D02204C330000E6
:105F90004C8D0220EE290000C40F0000C20D00004D
:105FA000962B0000C0B50000182B0000CC2A000082
:105FB00010B50000FC2C000051ED8764309D0010EE
:105FC000D15F0010ACA4001024A50010E0A40010C4
:105FD00007B56046002800D100BE01880A0A0230D9
:105FE000DF2AFAD1C9B2820804D3028840880004AB
:105FF000104300E00068024A5050039007BD0000C3
:10600000508D022001480421014B1847D004002084
:10601000D9500010014B1B6818470000D004002025
:10602000014B5B6818470000D004002010B5030046
:10603000080011001B68984710BD0000F8B5070064
:106040000D001600437C002B02D0002400200CE041
:1060500003681100280098472DE03B7C10E00221E6
:1060600015483B689847601C0134B44214DA002C90
:10607000F3DD2B19013B1B780D3B5A425341DBB238
:106080002A5D0A2AF0D1002BEED1A042E7DA211ACC
:1060900028183B689847E2E7B04203DA311A28181B
:1060A0003B689847002E06DDAD19013D2B780D3B6E
:1060B0005A4253413B74F8BD24A6001070B5050048
:1060C0000368002B16D00C4B1C6805E0290004C99E
:1060D0002000FFF7B3FFE468002C09D02368002BF1
:1060E000F9D0064B1B68002BF0D0A342F3D1EDE7AB
:1060F00000232B6070BDC0467C8702208087022071
:1061000070B505000C000B68802B05D021684B1C76
:1061100023606418257170BD0800FFF7CFFFF5E715
:10612000F0B583B007000E000092019328E0A36849
:10613000002B04D0310038009847002827DCE468A1
:10614000002C06D0134B1D68002DF0D0A542F6D1CF
:10615000EDE701200021FCF7D9FE0099019A0E4BD2
:106160005B6A9A4209D80C48806A88420BD29A42EC
:1061700001D0012302E0002300E00023002B04D122
:10618000064B1C68DCE70123F8E70120404203B01E
:10619000F0BDC04680870220004005407C87022079
:1061A00010B582B0D0231B0600241C5701A9074854
:1061B00003F06AF9002806D1019B9C4203D00348F2
:1061C00003F072F9012002B010BDC046280500207E
:1061D00010B5024803F040F910BDC0462805002064
:1061E000F0B5CE46474680B583B006000D00904618
:1061F0001C00FFF7D5FF81466B1C05D0002C08D092
:10620000194F1A4B1C6807E0300003F0EDF8050049
:10621000F4E7174FF5E7E468002C17D02368002B4C
:10622000F9D0144B1B68002B01D0A342F3D12A00F4
:1062300031002000B8474346002BECD06B46D91DF7
:106240000A230B7001222000B847E4E74B46002BDD
:1062500007D16B1E9D41E8B203B0C0BCB946B04641
:10626000F0BDFFF7B5FFF4E72D6000107C8702203A
:106270003D6000108087022010B582B004006B469C
:10628000D81D0470012300220121FFF7A9FF20007F
:1062900002B010BD094A01E00C331A001368002B4C
:1062A00008D08342F8D1002907D1C36813600023C6
:1062B000C36002E0002900D0106070477C87022094
:1062C00010B5064B1C6801E09847E468002C03D029
:1062D0006368002BF8D1F8E710BDC0467C87022028
:1062E00070B5050003F080F80400002301220100CE
:1062F0002800FFF775FFFFF7E3FF200070BD0000E7
:1063000070B5A2B004000E00FFF74AFF050084221A
:10631000002101A8FFF77EFE3300220001A90848F2
:10632000FEF7B2FE040001A8FFF7C8FEFFF7C8FFA2
:10633000002D02D1200022B070BDFFF749FFF9E720
:10634000016100100FB400B583B004A901C9019127
:10635000FFF7D6FF03B008BC04B0184710B500F033
:1063600073F910BD30B583B004000025FCF7AEFD15
:1063700002000B1E16DB12196B41994202D804D1A0
:10638000904202D901225242D317002B10DB012187
:1063900001A8FFF7C5FE002802DB0FD001AB18787B
:1063A00003B030BD094B0A4A3F210A48FDF7FCF80B
:1063B000064B074A3F210748FDF7F6F89221064BA6
:1063C000064A49000648FDF7EFF8C0464498001019
:1063D000F8A50010609800107099001010A6001029
:1063E000BCA5001070470000014B00221A707047D6
:1063F0009A8E02204B79FF2B0CD18B79002B0BD17D
:10640000CB79012B0AD1082A0AD98A78054B1A7050
:10641000092000E0002070470020FCE70020FAE798
:106420000020F8E79A8E02200120704770B5040022
:106430000D000348FEF740FE0300290020009847A6
:106440005542000010B5002926D1117953791B025D
:106450000B43124909788B4201D0002010BD5378BC
:10646000012B03D0022B10D00020F7E79178D378CE
:106470001B021943DB0503D54B0A0120984000E0BD
:1064800000207F231940FFF7D1FF64220021002064
:10649000FDF732FD0120E1E70120DFE79A8E0220BF
:1064A000012303700048704728A6001010B50B7830
:1064B0004878000218438A7812041043CB781B06F0
:1064C00003439622D200934200D010BD0021080061
:1064D000FFF7ACFF30B583B005000C0001A91848E8
:1064E00002F0D2FF002808D1D0231B061B68019AB6
:1064F0009A4221D0124802F0D7FF002001F01AFE84
:10650000002807D1032464420D4802F0A5FF2000B3
:1065100003B030BD002001F02FFE002802D103247B
:106520006442F1E722002900002001F031FE041E40
:10653000EAD103246442E7E703246442E7E7C04664
:106540005C8E022010B50021054802F09DFF002856
:1065500000D110BD01F086FB014802F07DFFF8E795
:106560005C8E0220F0B5C64600B582B080460D00B4
:1065700001A92E4802F088FF002808D1D0231B066D
:106580001B68019A9A420FD0284802F08DFF002024
:1065900001F0D0FD002847D1254B002000211860D4
:1065A0005960224802F058FF02B080BCB846F0BDE6
:1065B00001F058FB002001F0FFFD002001F0BAFDC2
:1065C0000028EED0002001F079FE00281DD0AC425A
:1065D000E7DA2E1B002001F071FE0200864200DC8B
:1065E0003200002AE4D043461919002001F04AFE87
:1065F000060001F037FB002001F0DEFDA419FCF7D6
:1066000065FC0B4B18605960E1E7FCF75FFC084B39
:106610001E685F68074A002392197B419942C0D8DF
:10662000D5D19042D3D9BCE70024D0E75C8E0220BC
:106630000081022020A1070010B51F20FDF7EAF914
:10664000FA208000002110BD70B584B0244B1B7867
:1066500002F07AF823491F20FDF7ECF901211F20F1
:10666000FDF7D0F92048FCF759FDFCF7A3F9060027
:10667000FCF72CFC04000D1E20DBFA229200002304
:1066800012196B41994202D804D1904202D90122D9
:106690005242D317002B17DB0121029100210191F7
:1066A000124900913000FCF79BF90400631E9C41E5
:1066B000E4B200280ED1200004B070BD0C4B0D4A8E
:1066C0003F210D48FCF770FF094B0A4A3F210A4859
:1066D000FCF76AFF01210948FFF7DCFDEBE7C04644
:1066E00094AE0010456500105C8E022039660010E3
:1066F0004498001060A6001060980010E00400208C
:1067000000487047F8A6001000487047A4A6001083
:1067100010B50400154B1B78002B0ED0002C11D1A6
:10672000134B144A5A80012301335B001BB2C02271
:10673000920013430E48038010BD11210B4802F054
:10674000D7FBEBE7052C0ED8A4000B4BE458002335
:10675000122BE9D8E25C002AE6D001335900044844
:106760004252DBB2F4E70020E6E7C0467C8E02200E
:1067700044870220090400000CA7001002007F20BB
:106780001040D209400080184001014BC0187047EA
:106790008487022010B582B001AB074A1A8000241A
:1067A00006E001AB185DFFF7E9FF0123C370013478
:1067B000012CF6D902B010BD0080FFFF10B5838B0D
:1067C0003F333F229343022915D0124C2268C26006
:1067D000D31823609C0610D10F4C62406340802484
:1067E0006401A3420FD88906114380231B06194375
:1067F0004368196010BD5B00E7E7084B084A542165
:106800000848FCF7D1FE084B054A56210548FCF71D
:10681000CBFEC0462C8C02200000105024A7001094
:106820003CA8001054A70010A8A70010F8B5050058
:106830000E001400FFF7A2FF7F232B40EF098570A5
:106840007A427A4142700022C27086838477012F97
:106850000DD0DA0012498C466244826082680021C1
:106860001160002B09D143600E4BC360F8BDDA0004
:106870000D498C4662448260F0E7012F09D0013B4C
:10688000DB000A4A9446634443602100FFF796FF09
:10689000ECE7013BDB00064A944663444360F4E7BF
:1068A0008400105000011050800010500C00105057
:1068B0000800105010B5002308E00133DA00002171
:1068C00008481150844662445160DBB20E2BF4D963
:1068D000F022920000210448FFF79CFB034B044A7E
:1068E0001A6010BD00001050C48702202C8C0220BA
:1068F00080011050F0B5CE46474680B583B01D4BA1
:106900009F6D0024012603E0B74376000134E4B212
:10691000002F29D01F2C27D83E42F6D0164B9E655B
:10692000630899460123634001221A4090464B4672
:106930005D0045446D01114BED18280000F0ACFAE4
:106940000028E1D04B465B0043445B010B4AD3185F
:106950009A8A9978012300930023002000F00AFE10
:10696000280000F009FACFE703B0C0BCB946B04632
:10697000F0BDC04600001150003011508487022045
:1069800070B52B4A9823D45880235B0225001D4004
:106990001C420AD1E30616D4E30419D4630429D4B3
:1069A000230433D4A5423ED170BDFFF7F3FE01228C
:1069B0002049002000F0C4FD1F4B802292021A657E
:1069C00080256D02E6E710231D43FFF793FFE3E701
:1069D00080235B011D43164B00221A60FFF76AFFFC
:1069E00001220021002000F096FD134B80221203AB
:1069F0001A65D3E78023DB011D4301220421002017
:106A000000F076FD0C4B10221A65C9E780231B02AB
:106A10001D4301220521002000F06AFD064B802263
:106A200012011A65BEE7290061400448FCF756FED2
:106A3000000011500000105000301150DCA7001071
:106A400070B50C001500FFF799FE2A00210000F038
:106A5000FFF970BD10B5002804D101210520FCF715
:106A6000D1FF10BDB921034B034A49000348FCF78D
:106A70009BFDC046F0A700102CA8001054A70010E2
:106A800010B5002805D1002200218020FFF7D8FF93
:106A900010BDBF21024B034A49000348FCF784FDA7
:106AA000F0A700101CA8001054A70010024B802271
:106AB0005202DA647047C0460020115070B5041EBF
:106AC00025D100F033F9154D0C23AB67144905208F
:106AD000FCF7B0FF402200211248FFF79BFA00228A
:106AE00040210020FFF7A2FE002240218020FFF776
:106AF0009DFEFFF7DFFE01232B6480239B05EB64E3
:106B00009023094AEA502000FFF7D0FF70BD4E21C4
:106B1000064B074AFF310748FCF746FD00001150BD
:106B2000816900108487022010D00100F0A70010B6
:106B300050A8001054A700100B785B0602D14B78C8
:106B4000052B00D070478A78014B1A60FAE7C046DF
:106B50000000115010B50C0000280DD10A794B79B6
:106B60000721194009021143E2789207920FA07899
:106B7000FFF75CFE012010BDD621034B034A4900FC
:106B80000348FCF711FDC046F0A700100CA8001048
:106B900054A7001010B5FFF78DFE10BD10B504000E
:106BA000080011001A00002C03D1FFF749FF012053
:106BB00010BDBC21024B034AFF310348FCF7F4FC33
:106BC000F0A70010FCA7001054A7001010B5080093
:106BD0004B0605D1CB09012B0AD00222054B9A6640
:106BE000FFF7CCFD80221201002100F0CBF810BD90
:106BF0000122F3E70020115010B508004B0600D128
:106C000010BDFFF7BBFD0023C3700022014900F057
:106C1000B9F8F5E7FFF7FFFFF8B504000F00438A66
:106C2000828B1E1C934200D9161CB6B29B1B63823A
:106C30008025ED003543E378002B13D080229201AC
:106C4000154301225340E3706378002B0CD0638A14
:106C5000002B02D18023DB011D43002F00D02D0427
:106C60002800F8BD0022EBE7B801E3689C466044C9
:106C70003200A169FFF7D4F9A3699C466644A66176
:106C800080231B021D43E2E770B5040083681B6884
:106C9000002900D01B0C9D05AD0D6278002A11D192
:106CA0001B0409D4A38A5B19A382A38BAB4201D92D
:106CB00000236382280070BD0E4B0F4AD7210F4876
:106CC000FCF772FC1B040ED58901E3689C46614405
:106CD0002A00A069FFF7A4F9A38A5B19A382A3691C
:106CE0005B19A361E1E7064B034ADE210348FCF789
:106CF0005BFCC0465CA800107CA900107CA80010BA
:106D0000D0A8001010B5040083681B680021FFF7AD
:106D1000BBFF63681B685B0002D5A38B834200D076
:106D200010BD01212000FFF7AFFFF9E710B5802368
:106D30005B040C4A13600C4A13600C4B9A68802366
:106D40005B049343F9D10A4C9C2200212000FFF7F9
:106D500061F98022520100210648FFF75BF90923FF
:106D6000636710BD00E0004000F0004000C000403C
:106D700000001150000010500023037443828382EE
:106D80008361704710B5002902D083681B681940E1
:106D9000002A0FD0114353050CD5826813685B0598
:106DA0000BD40B4B0B401360FFE7FFE7FFE7FFE758
:106DB000FFE7FFE78368196010BD83787F211940E2
:106DC000DB099B00034A9A580348FCF787FCC0463E
:106DD000FFFBFFFFF4040020F0A8001070B50400D2
:106DE00043681E680021FFF717FF80256D010543EA
:106DF000144B1B6C9B0704D4A378DB0914D101331B
:106E000000E00023628A002A01D0002B0ED00E4B36
:106E10001E4080239B053343626813602A000021D3
:106E20002000FFF7AFFF70BD0023EBE7012120003A
:106E3000FFF7F2FE0543054B1E40A023DB0533435D
:106E4000EAE7C04600001150FFFFFFAFFFFFFFDF82
:106E500070B504000D001600037C002B09D166827A
:106E60000023A38201332374A5612000FFF7B6FF3E
:106E700070BD83787F211940DB099B00044A9A5832
:106E80000448FFF75FFA2000FFF776FFE7E7C04608
:106E9000F404002010A9001070B50400057C002D3A
:106EA00006D0FFF72FFF638A002B08D1280070BDA2
:106EB00081787F231940044A0448FCF70FFC200026
:106EC000FFF78CFF0025F1E7F404002048A900102B
:106ED00070B5050000240EE063001B19DA00184BA2
:106EE0001B689B1802E0230010E000235B68280069
:106EF00098470134E4B2134B1B78A3420ED3124AD5
:106F0000002AF0D0A342E7D8E31ADBB2002BECD181
:106F10005A00D218D2000D4B9B18E7E70C4C5322B5
:106F200000212000FFF776F8E01C1022FF21FFF778
:106F300071F8200013302022FF21FFF76BF870BD9D
:106F400064810220908E0220A1640010C4AA001067
:106F50009C84022010B5FFF7BBFF01F02BF810BD99
:106F600070B505000C001600C86801F02DF8E36844
:106F7000320000212800984770BD0000F0B5DE46C1
:106F800057464E464546E0B583B081460139C8B202
:106F9000FFF7BAFB002803D043789846022B0CD0A9
:106FA000564A57495748FFF7CDF9002003B0F0BCC7
:106FB000BB46B246A946A046F0BDC5796A11012379
:106FC00051491A4014010A781026B24322430A702C
:106FD000AD112B405B01D2B22024A24313430B70AE
:106FE000070009378178C3781B020B4382469A4415
:106FF00063E0FB789B463B78FF1865E0434A4049D5
:107000004048FFF79FF90020D0E766003619F300EB
:107010003F4A1668F61802E0230017E000262A000F
:1070200039004846B36898470190082801D985423D
:1070300014D20134E4B2374B1B78A34239D3364A19
:10704000002AE9D0A342E0D8E31ADBB2002BE5D155
:107050005E00F318DB00314EF618E0E75B46012BCB
:1070600010D0002293451AD9BB789B18DBB2264971
:10707000C918C978FF290BD12349CB18DC7001321C
:10708000D2B2EFE7B268264B9A42EAD1C346E8E7AC
:10709000244A1B491B48FFF755F9002086E71A4888
:1070A0002300019D2A003900133001F0BBFBAC46E0
:1070B0006744184B1B78A3420ED3574514D27B78F4
:1070C0000B2B96D001239B467B78042B96D15346FD
:1070D000DD1BADB20024AEE7F32292000849094857
:1070E000FFF730F9002061E70F4B002B03D000E0E1
:1070F00000BF01205AE7012058E7C0467B0300008B
:107100008CAA00108CA900109C8402209603000019
:1071100064810220908E0220A1640010C4AA001095
:10712000D9830010BD0300000000000070B5050009
:107130000C00CB7888780F2B54D89A002F498A58A6
:107140009746FFF7DDFA020012232100280000F025
:10715000DDFE48E02A4B002B46D000E000BF0200D5
:107160008178C3781B020B432100280000F0CEFE7B
:1071700039E0022B10D0234B002B37D000E000BFAA
:107180000200002A0CD09178D3781B020B43210017
:10719000280000F0BBFE26E0FFF7B6FA0200F0E799
:1071A000194A1A491A48FFF7CDF800201BE0237945
:1071B000617909021943FFF7ABFA021E18D0037870
:1071C0002100280000F0A2FE0DE0124B002B11D090
:1071D00000E000BF021E0FD003782100280000F05D
:1071E00095FE00E0002070BD0020FCE70020FAE7DB
:1071F0000020F8E70020F6E70020F4E7A4A900103B
:1072000000000000000000001404000074AA001038
:107210008CA9001000000000024B5878431E9841D2
:10722000C0B270479C840220024B18784007C00F00
:107230007047C0469C840220014B18787047C046B6
:10724000918E022070B50500274B1878002800D0D9
:1072500070BD532200212548FEF7DCFE244C20009F
:10726000FBF75CFF234B1C60234C20001C30FBF71A
:107270007BFF200001F0F0FD204B1C60204B002B19
:1072800004D02048FFF70CF91F4B186000240DE0D4
:1072900063001B19DA001C4B1B689B1802E02300DB
:1072A0000FE000231B6898470134E4B2154B1B78AC
:1072B000A3420ED3124A002AF1D0A342E8D8E31A1F
:1072C000DBB2002BEDD15A00D218D2000F4B9B1825
:1072D000E8E72800FFF7F2FB2800FFF7BBFB024BB3
:1072E00001221A700120B3E7918E02209C840220B3
:1072F00054840220F0840220FC040020F484022044
:10730000A1640010908E022064810220C4AA0010A3
:1073100030B585B004004378042B00D196E038D80E
:10732000022B62D0032B00D0B9E06D4B1B785B07BA
:1073300000D483E06A4A137804218B4313700C2233
:10734000002101A8FEF766FE23786A461371052323
:107350005371644B1C68E269EFF3108172B61368D5
:10736000002BFCD0BFF35F8F216201A9200001F048
:1073700038FDE269236ABFF35F8F0021116083F358
:10738000108800285AD1A82257495848FEF7DAFF3A
:1073900054E0052B00D082E0514B1B78DB074DD524
:1073A0004F4A137804218B4313704E4B1D68EA69D2
:1073B000EFF3108172B61368002BFCD0BFF35F8F20
:1073C00029622100280001F00CFDEA692B6ABFF355
:1073D0005F8F0021116083F3108800282ED1A8222E
:1073E00041494248FEF7AEFF28E03D4B1A780121A3
:1073F0008A431A701A7801318A431A7000225A702F
:107400001A7802318A431A70364B1D68EA69EFF325
:10741000108172B61368002BFCD0BFF35F8F296216
:107420002100280001F0DDFCEA692B6ABFF35F8FC1
:107430000021116083F31088002801D005B030BD11
:10744000A82229492948FEF77DFFF7E7244B1B783E
:10745000DB07F3D5224A137804210B431370214B29
:107460001D68EA69EFF3108172B61368002BFCD037
:10747000BFF35F8F29622100280001F0B2FCEA69A6
:107480002B6ABFF35F8F0021116083F310880028FF
:10749000D4D1A82214491548FEF754FFCEE7114B6A
:1074A0001D68EA69EFF3108172B61368002BFCD0F7
:1074B000BFF35F8F29622100280001F092FCEA6986
:1074C0002B6ABFF35F8F0021116083F310880028BF
:1074D000B4D1A82204490548FEF734FFAEE7C04600
:1074E0009C840220F484022064AA00108CA900105D
:1074F00070B584B006000D0014000C22002101A814
:10750000FEF788FD6B461E715D71210001A8FFF733
:10751000FFFE04B070BDF0B585B007000E00150089
:1075200001AC0C2200212000FEF774FD277001231E
:107530006370267129002000FFF7EAFE05B0F0BD58
:1075400070B584B006000D0014000C22002101A8C3
:10755000FEF760FD6B461E7106236A4653710822D2
:10756000290002A8FEF75CFD210001A8FFF7D0FE6C
:1075700004B070BDF0B5CE46474680B585B08046B4
:107580000F0016001D000CAB1B78994601AC0C22B5
:1075900000212000FEF73EFD434623700723637061
:1075A00027710396657149462000FFF7B1FE05B0CB
:1075B000C0BCB946B046F0BD70B506000D008B7872
:1075C00070221A420DD10D4B9978280001F0D6F89F
:1075D000041E0DD029003000FFF7BCFA0400200083
:1075E00070BD074A07490848FEF7ACFE0024F6E7DD
:1075F000064A04490448FEF7A5FEF0E79C840220F1
:10760000C204000040AA00108CA90010C3040000AE
:10761000F0B5D6464F464646C0B581460C00170029
:107620009846089B9A46002516E0184A18491948BA
:10763000FEF788FE00263000E0BCBA46B146A846F8
:10764000F0BD154A12491348FEF77CFEF3E7099A8C
:1076500013702378E4180135AF4214DD6378052BED
:10766000E3D1E1788907890F4145DED12100484601
:10767000FFF7A2FF061EE4D0A378DA09012AE6D0BC
:1076800052461370E5E70126D5E7C0469C0400008A
:1076900050AA00108CA900109D04000070B57F2531
:1076A0000D40CC096A001E4B9B181B193033DB7848
:1076B000DB07DE0F002B30D1194B9B181B19303321
:1076C000DB785B072AD4174B18680121494201F087
:1076D000E3FE6A00124B9B181B193033DB78DB0783
:1076E00008D40F4B9B181B193033DB785B0712D57E
:1076F000002600E00026002E08D06D0008494D1934
:107700002C193034E37804221343E370054B1868D6
:1077100001F0A2FE02E00126EDE70026300070BD78
:107720009C840220F084022070B57F250D40CC0996
:10773000154B18680121494201F0AEFE6A00134B57
:107740009B181B193033DB78DB0708D40F4B9B18D1
:107750001B193033DB785B0713D4002600E00026CA
:10776000002E08D06900094D6D182C193034E378CB
:1077700004229343E370044B186801F06DFE30005F
:1077800070BD0126ECE7C046F08402209C840220F4
:10779000F0B5C64600B582B001937F250D40CE09F5
:1077A0006F00174CE419A4193034E478E4071DD4B1
:1077B0006F00134CE419A4193034E3780127BC4658
:1077C00067463B43E370019BFFF7E8F9002813D1BC
:1077D0006D000B4B5D19AE193036F37801229343DF
:1077E000F370F37803329343F37005E0054A0649DA
:1077F0000648FEF7A7FD002002B080BCB846F0BDE9
:107800009C8402200A05000030AA00108CA90010F8
:1078100070B57F240C40CD0962000C4B9B185B199E
:107820003033DB789B0700D570BDFFF7CFF96300DD
:10783000064CE41864193034E37802221343E370F1
:10784000E37801221343E370EEE7C0469C840220F4
:1078500070B57F240C40CD0962000C4B9B185B195E
:107860003033DB789B0700D470BDFFF7C5F96300A8
:10787000064CE41864193034E37802229343E37031
:10788000E378013A9343E370EEE7C0469C8402201C
:107890007F220A40CB09520003498918C9183031A8
:1078A000C8788007C00F70479C840220F0B5C64698
:1078B00000B582B005000C00002000F085FB2378A5
:1078C00060221340602B12D0402B17D02278D206B2
:1078D000D20E012A00D1D9E0022A00D120E1002AEB
:1078E0001AD00026300002B080BCB846F0BDCC4AA9
:1078F000CC49CD48FEF726FD0026F3E7CB4B002B05
:1079000000D181E1180000F05FFB22000021280077
:1079100000E000BF0600E5E7202B0AD0002B00D0D6
:107920007AE16378092B00D978E19B00C04AD358EB
:107930009F4623790F2B00D968E1BE4AD318DB7824
:10794000BD4A002A05D0BD4A1278934212D39B1A31
:10795000DBB2002B00D05BE15900CB18DB00B8494B
:10796000C918002900D155E122002800FFF7F8FAD4
:107970000600B7E75900CB18DB00B24A1168C918F6
:10798000EFE7200000F026FBA1782800FFF778F849
:10799000A84A137802210B4313700126A2E7A54BD6
:1079A0005B786A460632137001232100280000F03C
:1079B000ADFA012696E7A7789E4B5B78DBB2BB4217
:1079C00005D09C4B5B78002B09D1002F13D1994B2C
:1079D0005F702100280000F07DFA012682E7280070
:1079E000FFF7D8F8934EB37898462800FFF770FA5F
:1079F0004346B370E9E739002800FFF7BFFA061ED7
:107A0000E5D1914A87498848FEF79CFC6AE7210046
:107A10002800FFF78BFB060064E7A278E3781B02DF
:107A20001343012B01D000265CE7824A137808211A
:107A30000B4313702100280000F04CFA012651E797
:107A4000A278E3781B021343012B01D0002649E7FB
:107A5000784A137808218B4313702100280000F026
:107A600039FA01263EE7734B1A785109920801232F
:107A70000B4002210A4013436A4606321380022358
:107A80002100280000F042FA01262BE723790F2B72
:107A900000D9DDE0674AD318D978674B002B05D0B1
:107AA000664B1B78994229D3C91AC9B2002900D064
:107AB000D0E04B005B18DB006149C918002900D1F8
:107AC000CAE022002800FFF74BFA061E00D009E7A3
:107AD000237860221A4200D004E763780A3B012B26
:107AE00000D9FFE6002000F06FFA63780A2B0CD073
:107AF0002100280000F0EEF90126F3E64B005B18A8
:107B0000DB00504A1168C918D8E76B469A1D00235C
:107B1000137001332100280000F0F8F90136E1E686
:107B200021797F220A40CE097020084220D15200DC
:107B3000404882189219D27C3F48002805D03F481F
:107B4000007882421BD3121AD2B2002A1ED15600EC
:107B5000B218D2003A4EB618002B19D0002E00D120
:107B60007CE0220031002800FFF7FAF90600B9E6B0
:107B7000364A2C492C48FEF7E5FB0026B2E65600B3
:107B8000B218D2002F480668B618E5E70026E3E7EA
:107B90006378012B12D0032B10D0002B01D00026CC
:107BA000A0E62800FFF774FE6B469A1D10800223A2
:107BB0002100280000F0AAF9012693E6A778E278D0
:107BC00012023A4304D1012B1AD02800FFF720FEFD
:107BD000002E45D0220031002800FFF7C1F9002017
:107BE00000F0F2F9134A3423D35CDB07DE0F002BDD
:107BF00000D077E62100280000F06CF9012671E63C
:107C00002800FFF725FEE3E700266BE6002669E67D
:107C1000002667E6002665E6002663E6002661E6A4
:107C20007F020000A0AA00108CA900100000000034
:107C3000E4A900109C840220A1640010908E022010
:107C4000C4AA001064810220D302000033030000A4
:107C5000002647E6002645E6002643E6002641E6E4
:107C600001263FE630B585B000F080FD002808D140
:107C700005B030BD01AC2078FFF76CF92279724B6A
:107C80009A70724B1C68E269EFF3108172B6136848
:107C9000002BFCD0BFF35F8F216201A9200001F00F
:107CA0007AF8E269236ABFF35F8F0021116083F3E2
:107CB00010880028DCD001AB5B78082BE1D89B0052
:107CC000634AD3589F4601AB1878FFF743F9614BDD
:107CD000002BD6D000E000BFD3E75B4B1A7801241D
:107CE00001210A431A703322995CA1439954995C8B
:107CF0000420814399540132995CA1439954995CC1
:107D00008143995401AB187802A9FFF7CFFD0028F1
:107D1000B7D101AC20780021FEF758FF20788021F0
:107D2000FEF754FFADE701AB19797F220A40CC0979
:107D30005000454B1B181B193033D8780125A84338
:107D4000D870D8780335A843D870002A1DD05200C7
:107D50003D4B9A181219D37C3F4A002A05D03F4A5E
:107D60001278934218D39B1ADBB2002B1BD15A0016
:107D7000D218D2003A4B9B18002B14D01C6901A8D2
:107D80004279039B0078A0477BE701A84279039BD7
:107D9000007800F02DF974E75A00D218D200314B68
:107DA0001B689B18E8E7304A30493148FEF7CAFAA9
:107DB0005EE7254B1B78DB0700D462E72D4B002BD9
:107DC00000D15EE7204B18780007C00F00E000BF2D
:107DD00057E71D4B1B78DB0700D452E7264B002BDF
:107DE00000D14EE700E000BF4BE763001B19DA004B
:107DF0001C4B1B689B1802E0230014E000235B6906
:107E0000002B02D001AA107898470134E4B2134B3A
:107E10001B78A34200D234E70F4A002AECD0A342D9
:107E2000E3D8E31ADBB2002BE8D15A00D218D20013
:107E30000B4B9B18E3E70024E9E7029B002B00D1E2
:107E40001FE7039898471CE79C840220F4840220D3
:107E50000CAA001000000000A1640010908E022007
:107E6000C4AA00106481022037020000B8AA0010E2
:107E70008CA900100000000000000000F8B505000B
:107E8000124B9F89DE89B91B89B20B1C402900D98E
:107E900040239CB20D4B1B785BB2002B08DB00210A
:107EA000B74211D00A4A23002800FFF771FCF8BD41
:107EB000B74201D18021F3E7044B996822000448BE
:107EC000FEF7AEF88021EBE70022ECE740840220C9
:107ED0005C84022070B506000C000B4D08222800BF
:107EE000FEF79EF80023AB60EB81AB810023E356E5
:107EF000002B06DB8021002300223000FFF748FC26
:107F000070BD0021F7E7C04640840220F0B5C646A8
:107F100000B580460C0016001D00234F08223800D3
:107F2000FEF77EF8BE600023FB81A379E1790902A8
:107F300019430B1CA94200D92B1C99B21A4A9381F0
:107F4000A279E3791B02134319D0002901D0002E36
:107F500008D04046FFF792FF041E0AD0200080BCE4
:107F6000B846F0BD732211491148FEF7EBF9002421
:107F7000F4E779220D490E48FEF7E4F9EEE7002315
:107F8000E356002B0DDB8021002300224046FFF743
:107F9000FFFB041EE2D17E2204490548FEF7D2F918
:107FA000DCE70021F0E7C04640840220F4AA00107C
:107FB0008CA9001010B5142200210248FEF72AF8FF
:107FC00010BDC04640840220014B18617047C04676
:107FD0004084022010B50100044C08222000FEF766
:107FE0001FF80023A360E381A38110BD4084022019
:107FF00070B505001C00C909374B1B78DB098B42A3
:1080000019D0002C10D1354B002B02D03249FEF78D
:1080100093FD314B1B69002B03D02F4A022128000E
:1080200098470124200070BDAB222D492D48FEF752
:1080300089F90024F6E7284B1B785BB2002B07DB9D
:10804000254B9868002844D022002749FDF7E8FF17
:10805000214AD3891B199BB2D38191680919916078
:10806000D288934201D03F2C28D81B4B1B69002B90
:1080700005D0194A012128009847002814D0164B32
:108080001B785BB2002B0DDB80210023002228002F
:10809000FFF77EFB041EC5D1D82211491148FEF717
:1080A00051F9BFE70021F0E700212800FEF78EFD1F
:1080B00080212800FEF78AFD0124B3E72800FFF79E
:1080C000DDFE041EAED1E32205490648FEF73AF96B
:1080D000A8E70024A6E7C04640840220396B0010C0
:1080E000DCAA00108CA900105C84022070B504008A
:1080F00005001035280000F03EFE3F2800D870BD76
:10810000E1780020FFF7CAFA0028F8D0280000F034
:1081100032FE3F2808D996239B00E218E1784023DD
:108120000020FFF735FBEAE7E1780020FFF7FCFAD3
:10813000E5E7000010B50400FFF76EF800280CD149
:108140000022002A11D0B6239B0063430948C018BF
:108150000379DB070BD5012008E0FFF765F800285D
:1081600001D10122EDE70022EBE7002010BD002045
:10817000FCE7C0466881022010B5B6239B00584337
:108180001030024BC01800F0DBFD10BD68810220EA
:1081900070B5B6239B005843064BC51892B21030F9
:1081A000C01800F019FE04002800FFF79FFF200010
:1081B00070BDC0466881022070B50500FFF72CF83D
:1081C000002804D10023002B09D1002070BDFFF747
:1081D0002BF8002801D10123F5E70023F3E7B624AB
:1081E000A4006C432834244BE4180434200000F02D
:1081F000A7FD002801D10020E8E7B62292006A43DB
:108200001D4B9B1899780020FFF748FA002801D1F0
:108210000020DBE7B626B6006E43A6239B009C46F3
:108220006644154BF61840223100200000F0D4FDC2
:10823000041E15D0B620800068430F4D2D18A97874
:10824000230032000020FFF7A3FA002801D020000D
:10825000BCE7C82209490A48FEF774F80020B5E7D0
:10826000B62080006843044D2D18A9780020FFF740
:108270005BFA0020AAE7C0466881022024AB001008
:108280008CA9001070B50500B624A400444328341E
:10829000094BE418043492B2200000F0D8FD060027
:1082A000200000F04DFD3F2801D8300070BD2800AF
:1082B000FFF782FFF9E7C0466881022010B5B623B8
:1082C0009B0058432830034BC018043000F053FD86
:1082D00010BDC04668810220F0B5CE46474680B545
:1082E00083B0B622920000212848FDF793FE0026B5
:1082F000002E04D003B0C0BCB946B046F0BD234F39
:10830000B624A40074433D19FF236B7100239846E3
:108310001F4AEA8001222A81AB72EB7208232B7379
:1083200021004831C919F833994620001030C0198E
:108330004346009301334A4600F0C9FC210049310D
:10834000FF31C91920002830C019043001230093DF
:108350004A4600F0BCFC92239B00E3189946B944BE
:108360004846FAF7DBFE43466B624B46AB6294230A
:108370009B009C466444E4192000FAF7CFFE2C646D
:1083800043466B640136F6B2B2E7C046688102200C
:1083900000C2FFFF70B50025002D00D070BDB624CF
:1083A000A4006C430B4EA01905220021FDF732FEFC
:1083B00020001030801900F04FFD2834A419043437
:1083C000200000F049FD0121200000F06BFD013587
:1083D000EDB2E1E768810220F0B583B006004B7989
:1083E000022B68D18B79022B69D10023002B08D096
:1083F0000027002F13D08B783B700C780C190925BF
:1084000019E0B624A4005C432E48001980780028A7
:1084100002D00133DBB2E9E72A4FE719E9E78F22FF
:10842000520029492948FDF78DFF002544E02178B5
:108430004D19ADB264186378242B01D19542F6D959
:10844000052B09D06378042B02D163790A2B18D04D
:108450003800FFF74BFE2FE021003000FFF7ACF8AB
:10846000002806D0A3787B7022785519ADB2A418E5
:10847000E8E79922520014491448FDF763FF0025EC
:108480001AE021784D19ADB26118BB1C0193FB1C99
:108490000093022302223000FFF7BAF8002802D02E
:1084A0000E35ADB2D4E7A122520007490748FDF7C7
:1084B00049FF002500E00025280003B0F0BD00259D
:1084C000FAE7C0466881022018AB00108CA90010A2
:1084D000F8B51400127860231340202B00D07FE001
:1084E000444A0025002D00D07CE016782779637976
:1084F0001B023B439E4206D00135EDB2B6239B00E2
:108500009C466244EEE76378222B31D009D8202BB9
:1085100011D0212B03D1002923D0012061E00020BC
:108520005FE0232B05D1002949D002294CD001203E
:1085300057E0002055E0002903D0022908D001208F
:108540004FE0063207232100FFF7E0FC012048E05E
:10855000294B002B48D0911D2800FDF7A7FF0120D3
:108560003FE0063207232100FFF7D0FC012038E06E
:10857000002903D0022906D0012032E02100FFF7B4
:10858000A9FC01202DE0A178E3781B020B43012018
:10859000190001400E005C08044013714B42594120
:1085A000C9B22C32100000F07DFC144B002B1DD002
:1085B00022003100280000E000BF012011E021006E
:1085C000FFF788FC01200CE00D4B002B10D0A378A6
:1085D000E17809021943280000E000BF012000E013
:1085E0000020F8BD0020FCE70120FAE70120F8E7B1
:1085F0000120F6E768810220AD6400100000000051
:1086000000000000F0B5D64600B582B001900F0022
:1086100000930024002C0DD0002C19D1EB78BB4224
:108620001ED0AB78BB4255D00124200002B080BCE4
:10863000BA46F0BDB625AD0065433D4BED18EB786D
:10864000BB42E9D0AB78BB42E6D00134E4B2E1E70B
:10865000B022FF3237493848FDF774FE0024E4E7C2
:1086600010239A46AA4496239B00E9186B461A8861
:10867000504600F0ECFB314B002B1BD06B79FF2BED
:1086800018D0002600E00136009B9E4212D26A7983
:10869000AB19962189008C4663441B789A42F2D12B
:1086A000504600F060FB0028EDD16979200000E021
:1086B00000BFE8E7224B002B04D0504600F053FBEC
:1086C000002803D02800FFF711FDAAE7200000E0F2
:1086D00000BFF7E71B4B002B02D0200000E000BFDB
:1086E0002000FFF769FD002801D001249DE7280044
:1086F0002C3000F025FB002815D1009B002B14D056
:108700009B0601D0012490E7A9780198FEF7C6FFE7
:10871000041E01D1012488E7A978002300220198D2
:10872000FFF736F881E701247FE701247DE7C046A3
:108730006881022008AB00108CA900100000000026
:10874000000000000000000010B50020FEF77AFDD8
:10875000041E01D0200010BD292202490248FDF765
:10876000F1FDF7E750AB00108CA9001010B5FEF733
:1087700063FD002800D0012010BD000010B5027973
:108780004479072323401B021A43C3789B079B0F9E
:10879000022B16D0032B2ED0012B01D0002010BDB0
:1087A000022904D01C4B934204D30120F7E7802315
:1087B000DB00F8E7502219491948FDF7C3FD0020F6
:1087C000EDE7022903D0402A0ED80120E7E78023F5
:1087D0009B009A4201D10120E1E758220F4910483D
:1087E000FDF7B0FD0020DAE75C220C490C48FDF7EC
:1087F000A9FD0020D3E7022904D04023934204D3EB
:108800000120CCE78023DB00F8E76322034904481A
:10881000FDF798FD0020C2E7FF0300003CAB00100D
:108820008CA9001070B5002503E00E78AD19ADB22B
:10883000891995420AD24C78052CF6D18E787A3473
:10884000344064000419F609A355EEE770BD030037
:108850008A1890B2884202D39A89904202D95A89E2
:10886000801880B2704710B503008A4204D8881A75
:1088700080B29C89A04204D9891A89B25889081A01
:1088800080B210BD838801E0C91A89B28B42FBD93E
:1088900008007047F0B583B00600019111001F0079
:1088A000D41AA4B29A4202D24389E41AA4B2B58877
:1088B000A54205D22A003000FFF7D5FF30822C00F8
:1088C000002C02D1002003B0F0BD39003000FFF7CA
:1088D000D9FF3168F288504309180198FDF7A0FBD1
:1088E0000120F0E7F0B583B0060093080CE00B78A8
:1088F0004D782D021D438C7824042543CB781B062C
:108900002B43336004313B005F1EBFB2002BEED11E
:108910000333100018401A4201D103B0F0BD002308
:108920000193020001A8FDF77BFB019B3360F4E794
:10893000F0B5DE4657464E464546E0B583B00500E5
:108940008A460CA909788488E01A80B21C1B141985
:10895000A4B2EE8807007743BFB27443A4B2A34623
:1089600073432C68A0469844002908D001291AD0E6
:1089700003B0F0BCBB46B246A946A046F0BD90424B
:1089800005D3724341465046FDF74AFBF0E73A00F3
:1089900041465046FDF744FB2968380050445A468A
:1089A000FDF73EFBE4E7904206D3724392B24146A4
:1089B0005046FFF797FFDBE703233A009A439146BF
:1089C00041465046FFF78EFF43464B4403213A0091
:1089D0000A400F4230D00421891A89B2081C594537
:1089E00000D95846C7B2FF2101405846441AA1B2E7
:1089F0008B460021019101A804E01A780270013031
:108A00000A000133511EC9B2002AF6D1296804E0D8
:108A10000A78027001301F0001317B1EDBB2002F8B
:108A2000F6D15346019A1A605B46002BA0D05A46F5
:108A30005046FFF757FF9BE72968F5E7F0B585B08B
:108A40000500029103920AAA11880BAA17785C1AF2
:108A5000A4B28B4202D24289A41AA4B2AE88A64222
:108A600008D2320019002800FFF7FDFE2882298A6B
:108A700089B23400002C0DD0039B9C4200D31C0013
:108A80002800FFF7FFFE030000972200029928004C
:108A9000FFF74EFF200005B0F0BDF0B583B0040035
:108AA0000D0016001F008069002803D001214942F3
:108AB00000F0F2FCE3899BB2228A01970092320017
:108AC00029002000FFF7BAFF0500218A89B20200C1
:108AD0002000FFF7BCFE2082A069002801D000F032
:108AE000BBFC280003B0F0BD70B582B0160095083D
:108AF00009E00B6803701D0A45701D0C85701B0E84
:108B0000C370043025006C1EA4B2002DF1D10323E4
:108B100032001A401E4201D102B070BD0B680193B1
:108B200001A9FDF77DFAF7E7F0B5DE4657464E4658
:108B30004546E0B583B005008A460CA90878AC88A4
:108B4000E11A89B21C1B1419A4B2EE880F007743F6
:108B5000BFB27443A4B2A34673432C68A0469844A2
:108B6000002808D001281AD003B0F0BCBB46B2469A
:108B7000A946A046F0BD914205D3724351464046F6
:108B8000FDF74EFAF0E73A0051464046FDF748FA45
:108B90002868390051445A46FDF742FAE4E7914209
:108BA00006D3724392B251464046FFF79DFFDBE782
:108BB00003233A009A43914651464046FFF794FFFB
:108BC00043464B4403213A000A400F422ED0042171
:108BD000891A89B2081C594500D95846C7B2FF21E5
:108BE00001405846441AA1B28B465146096801918A
:108BF00001A904E00A781A70013102000133501E05
:108C0000C0B2002AF6D1286804E00A780270013167
:108C10001F0001307B1EDBB2002FF6D15B46002B1C
:108C2000A2D05A465146FFF75FFF9DE72868F5E757
:108C3000F0B5CE4600B584B004008946151E0393F6
:108C400043D04069002803D00121494200F024FCB0
:108C5000E789BFB2238A9BB2227A002A2AD1A2884E
:108C6000F91A89B29F4202D26389C91A89B2531A8A
:108C70009BB22E1C9D4200D91E1CB6B239002000AA
:108C8000FFF700FE0300039A0092320049462000DD
:108C9000FFF74AFF320039002000FFF7D8FDE081DE
:108CA0006069002801D000F0D7FB300004B080BC20
:108CB000B946F0BDA688AE4205D8AA1BE588554343
:108CC000A9441F00DAE72E00D8E71600EDE7F0B55B
:108CD00083B005000F001400019308AB1E788023B9
:108CE0001B029A4228D84069002803D0012149423A
:108CF00000F0D2FBA869002803D00121494200F00E
:108D0000CBFB2F60AC80019BEB802E726400013C9A
:108D1000A4B2AC81E4436C810023EB812B826869AF
:108D2000002801D000F098FBA869002806D000F0C8
:108D300093FB012003B0F0BD0020FBE70120F9E721
:108D400010B5C3899CB2028A91B29B1A9BB28C4225
:108D500002D242899B1A9BB28288101C9A4200D987
:108D6000181C80B210BD0300C0891B8AC01A434280
:108D70005841C0B2704730B5C3899DB2018A8CB2E8
:108D800082885B1A9BB2A54202D240891B1A9BB211
:108D9000D01A80B230BD70B504000D008069002883
:108DA00003D00121494200F077FBE28992B2238A85
:108DB0009BB229002000FFF76DFD0500218A89B2D2
:108DC00082B22000FFF743FD2082A069002801D075
:108DD00000F042FB280070BD10B50023FFF75DFED8
:108DE00010BD70B504000D004069002803D00121BA
:108DF000494200F051FBE3899EB2228A91B29B1A4C
:108E00009BB2B14202D962899B1A9BB2A2889A4254
:108E100002D1207A002817D031002000FFF732FD60
:108E2000E288504323689C4660442900FDF7F8F827
:108E3000012231002000FFF70AFDE081606900286F
:108E400003D000F009FB012070BD0120FCE710B544
:108E50000023FFF7EDFE10BD10B5040040690028A7
:108E600003D00121494200F017FBA069002803D07C
:108E70000121494200F010FB0023E3812382A388F3
:108E80005B00013B9BB2A381DB43638160690028E7
:108E900001D000F0E1FAA069002801D000F0DCFA6E
:108EA000012010BD70B504000D004069002803D0FA
:108EB0000121494200F0F0FAA069002803D0012105
:108EC000494200F0E9FA25726069002801D000F0FB
:108ED000C3FAA069002801D000F0BEFA012070BDDD
:108EE00010B5024800F034F810BDC046448C022092
:108EF00010B5002901D000230AE0114B114A1F319F
:108F00001148FAF751FB00240DE03732C254013307
:108F10004A1E9A420FD90F2B0DD85A080B4CA25C4F
:108F2000DC07F0D40424224114000F222240092A35
:108F3000EBDC3032EAE7C0180023037010BDC046F6
:108F40005CAB0010A8AB001064AB0010448C022096
:108F500070B588B0040004AD0026049609220021F3
:108F600005A8FDF757F800960922002101A8FDF792
:108F700051F84B232B700D226946280000F064FA4B
:108F8000002304E05A1D69468A5CE2540133072B32
:108F9000F8DD08B070BD000010B501000148F9F718
:108FA0005FF910BD8E8E022000B583B00100044B26
:108FB00000930B2300220348F9F729F903B000BD01
:108FC00030AD00108E8E02200523CB56002B01DB26
:108FD000934211D1094B9C46604443425841800062
:108FE000074BC058097901238B40013B934018403F
:108FF00043425841C0B270470020FCE70000D0AFA8
:10900000B885022070B50A79202A19D8174B9C46DA
:109010006044434258418000154BC458012393409B
:10902000013B497949B2002910DB08002025AA1A22
:10903000914218DC8B401C4201D00120404270BD9F
:109040000C4B0D4A40210D48FAF7AEFA2020801A49
:10905000002805DB1A0082401442F0D00138F7E7FF
:1090600001204042EBE701204042E8E70000D0AF9A
:10907000B885022050AD001054AE00107CAD001039
:1090800070B505000C001600FFF79EFF002801D008
:10909000002007E01548FAF721FB831912339B00E3
:1090A0005A510130237983420FD92378617809021C
:1090B0001943A27812041143E3781B060B434200C4
:1090C0009A5A530BE9D19219E7E701229A4013000B
:1090D000013B074A944665446A425541B340054AFC
:1090E000AD00A9580B43AB5070BDC046B8AD0010E1
:1090F0000000D0AFB885022010B5054B9C466044F7
:1091000043425841800041180248F9F7A9F810BDC0
:109110000000D0AF988E022010B582B00A4B9C465A
:109120006044434258418400E31C084A00922200F4
:109130000748F9F76CF8844202DC001B02B010BD4E
:1091400001204042FAE7C0460000D0AFCCAD00108D
:10915000988E0220F8B505000E00F9F729F80700EF
:1091600031002800FFF74EFF041E09DB020031002A
:109170002800FFF785FF3800F9F726F82000F8BD32
:109180000148FAF7ABFAC046B8AD001070B504005C
:109190000B7901259D40013D9540F9F709F80C4BED
:1091A000E3185A42534199000A4A8A58290011404B
:1091B000A94206D19B00AA4306495A50F9F704F880
:1091C00070BD054B054A8A210548FAF7EDF9C046FE
:1091D0000000D0AFB8850220F0AD001040AE001006
:1091E0007CAD001010B50400F8F7E2FF0A4BE3185D
:1091F0005A4253419B00094A00219950002306E03E
:109200001F2119401A0012329200115101331F2BF5
:10921000F6D9F8F7D9FF10BD0000D0AFB88502200D
:10922000F0B5CE46474680B581464B005B18DB0063
:109230004B44DC331B689C460027202417E0AE0615
:109240007B011E434B005B18DB004B44DC20804657
:109250009844404606601F261640B046E026360277
:1092600040460643D8331E60641B7F195209002C08
:1092700004D02500052CE2D90525E0E74B0059185C
:10928000C90049440800DC3063460360C0BCB946ED
:10929000B046F0BDF0B505AC25784C006418E4008C
:1092A0000419DC342468A446002D01D01F2614E0E4
:1092B000002612E05401A0256D0525434C006418DA
:1092C000E40004192700DC373D600D4D3543D834E8
:1092D0002560053B05321F242240052BEAD89B065A
:1092E000520113434C006218D20082181500DC357D
:1092F0002B60034B1E43D832166063462B60F0BDD3
:1093000080E00000F0B58BB004000D00160002688C
:109310000121A9408A430260002B35D06900491918
:10932000C90041180A00C832186810600432586831
:109330001060043298681060DB68DC310B606900F3
:109340004B19DB00D033E3188022520113438022F3
:1093500012061A601A60234BAB40A3602268281DD6
:1093600001231F0087403A4322602268280008300A
:109370008340134323601F2216404919C900641813
:10938000D83426600BB0F0BD1022002106A8FCF7EF
:1093900041FE80235B020693F8235B020793802340
:1093A000DB020893C0231B030893102206A902A81E
:1093B000FCF736FE6B005B19DB00E3181A00C832BD
:1093C00002991160039A01921A00CC32019911603E
:1093D000049A01921A00D03201991160059ADC3387
:1093E0001A60ACE70101010110B583070AD0030040
:1093F000032102E001330B4205D01A78002AF9D18B
:10940000181A10BD030019680C4A0D4C8A188A43BB
:1094100022420FD15968094A04338A188A432242EA
:1094200008D15968054A04338A188A432242F1D088
:1094300000E001331A78002AFBD1E1E7FFFEFEFECF
:1094400080808080F8B5C04601B40248844601BCE3
:10945000604700BF0503002001B40248844601BCF8
:10946000604700BF5102002001B40248844601BC9D
:10947000604700BFDD03002001B40248844601BC00
:10948000604700BFDD03002001B40248844601BCF0
:10949000604700BF0901002001B40248844601BCB6
:1094A000604700BFDD01002001B40248844601BCD2
:0894B000604700BFC10000206D
:1094B800636861696E5F746F203C3D204E554D5F57
:1094C800444D415F4348414E4E454C530000000017
:1094D800463A5C5069636F53444B5C5069636F5CF8
:1094E8007069636F2D73646B5C7372635C72703246
:1094F8005F636F6D6D6F6E5C6861726477617265D2
:109508005F646D615C696E636C7564652F68617218
:1095180064776172652F646D612E6800647265718D
:10952800203C3D20445245515F464F524345000080
:109538004552525F554E4B4E4F574E5F4D53470065
:109548004C4F4749435F414E414C595A45525F562B
:10955800315F3000434150545552455F5354415296
:1095680054454400434150545552455F4552524F6B
:109578005200000053797374656D20636C6F636BE0
:10958800206F66202575206B487A2063616E6E6FA8
:10959800742062652065786163746C792061636802
:1095A8006965766564000000B89500100CFF00003E
:1095B800A0802060A0804060C7201D40C7001D40DB
:1095C8004700404000C00B00D89500100BFF00007A
:1095D800A0802060A08040601D40C6001D4046005D
:1095E800404000C00A000000F89500100BFF000082
:1095F800A0802060A08040600040C4000040460079
:10960800404000C00A000000189600100BFF000040
:10961800A0802060A08040600040C6000040460056
:10962800404000C00A0000006368616E6E656C5FB0
:10963800636F6E6669675F7365745F636861696E9F
:109648005F746F006368616E6E656C5F636F6E66F2
:1096580069675F7365745F6472657100020304056E
:10966800060708090A0B0C0D0E0F1011121314151A
:10967800161A1B1C68775F69735F636C61696D6597
:109688006428626974732C206269745F696E64650A
:1096980078290000463A5C5069636F53444B5C502C
:1096A80069636F5C7069636F2D73646B5C7372635D
:1096B8005C7270325F636F6D6D6F6E5C686172644F
:1096C800776172655F636C61696D5C636C61696D1C
:1096D8002E63000068775F636C61696D5F636C651A
:1096E800617200004E6F207370696E6C6F636B73EC
:1096F8002061726520617661696C61626C65000049
:1097080072742D3E616C61726D5F6964203D3D200D
:1097180069640000463A5C5069636F53444B5C507F
:1097280069636F5C7069636F2D73646B5C737263DC
:109738005C636F6D6D6F6E5C7069636F5F74696D8C
:10974800655C74696D652E630000000069642026FD
:1097580026206964203C3D20706F6F6C2D3E686543
:1097680061702D3E6D61785F6E6F646573000000F7
:10977800256C6C642028686920253032782900001F
:109788006964202626206964203C3D206865617054
:109798002D3E6D61785F6E6F64657300463A5C506C
:1097A80069636F53444B5C5069636F5C7069636FA6
:1097B8002D73646B5C7372635C636F6D6D6F6E5C4D
:1097C8007069636F5F7574696C5C696E636C7564EE
:1097D800652F7069636F2F7574696C2F7068656188
:1097E800702E6800706172656E745F6964000000B5
:1097F8006368696C645F6964000000007061726589
:109808006E745F696420213D206368696C645F69D8
:10981800640000002170685F636F6E7461696E7325
:109828005F6E6F646528706F6F6C2D3E6865617040
:109838002C2072657573655F6964290075735F73A1
:10984800696E63655F626F6F74203C3D20494E54BA
:1098580036345F4D41580000463A5C5069636F5397
:10986800444B5C5069636F5C7069636F2D73646B04
:109878005C7372635C636F6D6D6F6E5C7069636F50
:109888005F626173655C696E636C7564652F70698E
:10989800636F2F74797065732E68000072656D6F41
:1098A8007665645F6964203D3D206E6578745F6904
:1098B8006400000063616C6C6261636B000000000F
:1098C800706F6F6C2D3E616C61726D5F696E5F7059
:1098D800726F6772657373203D3D206D616B655FC4
:1098E8007075626C69635F69642869645F68696739
:1098F800682C206E6578745F696429006964202685
:1099080026202170685F636F6E7461696E735F6E85
:109918006F646528686561702C20696429000000FF
:1099280064656661756C745F616C61726D5F706FA0
:109938006F6C5F696E697469616C697A65642829FE
:1099480000000000616C61726D5F696420213D2038
:10995800706F6F6C2D3E616C61726D5F696E5F70C8
:10996800726F677265737300726300004174746587
:109978006D7074656420746F20736C656570206900
:109988006E73696465206F6620616E206578636513
:109998007074696F6E2068616E646C65723B2075C7
:1099A800736520627573795F7761697420696620D1
:1099B800796F75206D75737400000000616C6172B9
:1099C8006D5F706F6F6C5F63616E63656C5F616C18
:1099D80061726D007570646174655F75735F73693A
:1099E8006E63655F626F6F7400000000616C617286
:1099F8006D5F706F6F6C5F616C61726D5F63616CDE
:109A08006C6261636B0000006765745F656E7472F9
:109A180079000000616C61726D5F706F6F6C5F67D9
:109A280065745F64656661756C7400006765745F72
:109A3800656E7472795F69645F68696768000000C1
:109A480070685F667265655F6E6F64650000000030
:109A580070685F6164645F6368696C645F6E6F649B
:109A68006500000070685F696E736572745F6E6F81
:109A78006465000070685F6765745F6E6F64650099
:109A88006164645F616C61726D5F756E6465725F5D
:109A98006C6F636B000000004861726477617265E7
:109AA80020616C61726D20256420616C726561644F
:109AB8007920636C61696D656400000074696D6587
:109AC800725F68772D3E696E747320262031752089
:109AD8003C3C20616C61726D5F6E756D000000002A
:109AE800463A5C5069636F53444B5C5069636F5CE2
:109AF8007069636F2D73646B5C7372635C72703230
:109B08005F636F6D6D6F6E5C6861726477617265BB
:109B18005F74696D65725C74696D65722E630000AF
:109B280068617264776172655F616C61726D5F73A1
:109B380065745F74617267657400000075706461B4
:109B480074655F75735F73696E63655F626F6F7469
:109B580000000000746F74616C000000463A5C50AD
:109B680069636F53444B5C5069636F5C7069636FE2
:109B78002D73646B5C7372635C636F6D6D6F6E5C89
:109B88007069636F5F73796E635C6D757465782E49
:109B9800630000006D74782D3E636F72652E7370DC
:109BA800696E5F6C6F636B006C6F636B5F69735F8B
:109BB8006F776E65725F69645F76616C6964286D42
:109BC80074782D3E6F776E65722900006D74782D5C
:109BD8003E656E7465725F636F756E740000000099
:109BE8006D757465785F6578697400006D75746566
:109BF800785F656E7465725F626C6F636B5F756EBC
:109C080074696C007570646174655F75735F7369FE
:109C18006E63655F626F6F7400000000726F6F742F
:109C28005F696400463A5C5069636F53444B5C500B
:109C380069636F5C7069636F2D73646B5C737263C7
:109C48005C636F6D6D6F6E5C7069636F5F7574696F
:109C58006C5C70686561702E630000002170685F3D
:109C68006765745F6E6F646528686561702C207223
:109C78006F6F745F6964292D3E7369626C696E67E2
:109C8800000000002170685F6765745F6E6F64652F
:109C980028686561702C20726F6F745F6964292D64
:109CA8003E706172656E7400666F756E64000000C8
:109CB8006E65775F7375625F7472656520213D20FC
:109CC800686561702D3E726F6F745F696400000093
:109CD80070685F72656D6F76655F616E645F6672EE
:109CE80065655F6E6F64650070685F72656D6F763D
:109CF800655F616E795F68656164000070685F61C7
:109D080064645F6368696C645F6E6F64650000001B
:109D180070685F6765745F6E6F6465002C20667598
:109D28006E6374696F6E3A2000000000617373659A
:109D38007274696F6E2022257322206661696C65D2
:109D4800643A2066696C6520222573222C206C6990
:109D58006E65202564257325730A000031203D3D7A
:109D6800202875696E747074725F74296C2D3E7347
:109D780070696E5F6C6F636B00000000463A5C5060
:109D880069636F53444B5C5069636F5C7069636FC0
:109D98002D73646B5C7372635C7270325F636F6D9A
:109DA8006D6F6E5C7069636F5F72756E74696D65F7
:109DB8005C72756E74696D652E6300000A2A2A2A22
:109DC8002050414E4943202A2A2A0A000A0000004E
:109DD80072756E74696D655F696E69740000000064
:109DE8007372635F66726571203E3D2066726571AD
:109DF80000000000463A5C5069636F53444B5C5066
:109E080069636F5C7069636F2D73646B5C737263F5
:109E18005C7270325F636F6D6D6F6E5C68617264E7
:109E2800776172655F636C6F636B735C636C6F63A0
:109E38006B732E6300000000636C6F636B5F636F6E
:109E48006E6669677572650064656C7461203E3D75
:109E5800202D323034382026262064656C74612029
:109E68003C3D203230343620262620212864656C7B
:109E78007461202620312900463A5C5069636F538B
:109E8800444B5C5069636F5C7069636F2D73646BDE
:109E98005C7372635C7270325F636F6D6D6F6E5C62
:109EA80068617264776172655F6972715C69727109
:109EB8002E630000212864656C7461203E3E2031C9
:109EC8003175290063757272656E74203D3D205F9F
:109ED8005F756E68616E646C65645F757365725FEB
:109EE800697271207C7C2063757272656E74203D86
:109EF8003D2068616E646C65720000006972715F74
:109F080068616E6465725F636861696E5F667265D9
:109F1800655F736C6F745F68656164203E3D2030D7
:109F280000000000767461626C655F68616E646C45
:109F38006572203D3D205F5F756E68616E646C657B
:109F4800645F757365725F69727100002128282843
:109F58002875696E747074725F7429767461626CA6
:109F6800655F68616E646C657229202D20282875EC
:109F7800696E747074725F74296972715F68616E5A
:109F8800646C65725F636861696E5F736C6F74732C
:109F980029202D2031292573697A656F6628737405
:109FA80072756374206972715F68616E646C657242
:109FB8005F636861696E5F736C6F742929000000C4
:109FC80030783163203D3D20282A696E7374293E1C
:109FD8003E31317500000000216578636570746951
:109FE8006F6E207C7C20657863657074696F6E2065
:109FF8003D3D206E756D202B2031360066616C73F7
:10A008006500000069735F7368617265645F6972F7
:10A01800715F7261775F68616E646C657228736CDA
:10A028006F745F68616E646C65722900657863653A
:10A038007074696F6E0000006972715F6164645FBB
:10A048007461696C5F746F5F667265655F6C697374
:10A0580074000000696E736572745F6272616E638A
:10A06800685F616E645F6C696E6B00006972715F36
:10A0780072656D6F76655F68616E646C657200000D
:10A088006D616B655F6272616E6368007265736FA4
:10A098006C76655F6272616E636800006972715FF9
:10A0A8007365745F6578636C75736976655F6861FD
:10A0B8006E646C65720000006662646976203E3DDD
:10A0C800203136202626206662646976203C3D20B1
:10A0D80033323000463A5C5069636F53444B5C50EE
:10A0E80069636F5C7069636F2D73646B5C73726313
:10A0F8005C7270325F636F6D6D6F6E5C6861726405
:10A10800776172655F706C6C5C706C6C2E630000BC
:10A1180028706F73745F64697631203E3D2031206A
:10A12800262620706F73745F64697631203C3D2069
:10A1380037292026262028706F73745F6469763269
:10A14800203E3D203120262620706F73745F64699D
:10A158007632203C3D20372900000000706F737470
:10A168005F64697632203C3D20706F73745F646968
:10A17800763100007265665F6D687A203C3D202864
:10A1880076636F5F66726571202F20313629000073
:10A19800706C6C5F696E697400000000666E69001F
:10A1A800666E692B000000006E616E00666E692D98
:10A1B80000000000124B0010C24A0010C24A0010F2
:10A1C8001C4B0010C24A0010C24A0010C24A0010BC
:10A1D800C24A0010C24A0010C24A0010C24A001007
:10A1E800084B0010C24A0010FE4A0010C24A001074
:10A1F800C24A0010F44A0010B44B0010DA4B0010A9
:10A20800F24B0010DA4B0010944B0010DA4B0010A0
:10A21800DA4B0010DA4B0010DA4B0010DA4B001062
:10A22800DA4B0010DA4B0010D04B0010DA4B00105C
:10A23800DA4B0010DA4B0010DA4B0010DA4B001042
:10A24800FE4B00102E5000104450001044500010D7
:10A258004450001044500010445000104450001066
:10A268004450001044500010445000104450001056
:10A278004450001044500010445000104450001046
:10A288004450001044500010445000104450001036
:10A298004450001044500010445000104450001026
:10A2A8004450001044500010445000104450001016
:10A2B8004450001044500010445000104450001006
:10A2C80044500010564E0010164E0010564E001006
:10A2D80044500010445000104450001044500010E6
:10A2E80044500010445000104450001044500010D6
:10A2F80044500010445000104450001044500010C6
:10A3080044500010445000104450001044500010B5
:10A318000A4C0010445000104450001044500010E3
:10A328004450001044500010445000104450001095
:10A3380044500010445000100A4C0010A64E001063
:10A348000A4C0010564E0010164E0010564E0010C3
:10A35800445000100A4C00104450001044500010A3
:10A368004450001044500010445000100A4C001093
:10A37800F84F001044500010445000101E4F0010B9
:10A38800445000100A4C0010445000104450001073
:10A398000A4C001000000000000000000000F03F20
:10A3A80000000000000024400000000000005940A8
:10A3B8000000000000408F40000000000088C340FB
:10A3C80000000000006AF8400000000080842E4170
:10A3D80000000000D01263410000000084D79741BC
:10A3E8000000000065CDCD412A282875696E7438B3
:10A3F8005F74202A29282828766F6964202A297200
:10A408006F6D5F646174615F6C6F6F6B75702872DC
:10A418006F6D5F7461626C655F636F646528275355
:10A42800272C202746272929292D322929202A2087
:10A4380034203E3D2053465F5441424C455F5632DE
:10A448005F53495A45000000463A5C5069636F53B0
:10A45800444B5C5069636F5C7069636F2D73646B08
:10A468005C7372635C7270325F636F6D6D6F6E5C8C
:10A478007069636F5F646F75626C655C646F756249
:10A488006C655F696E69745F726F6D2E63000000A2
:10A498005F5F61656162695F646F75626C655F6962
:10A4A8006E6974002A282875696E74385F74202ACA
:10A4B8002928726F6D5F7461626C652D32292920BD
:10A4C8002A2034203E3D2053465F5441424C455F8C
:10A4D80056325F53495A4500463A5C5069636F5398
:10A4E800444B5C5069636F5C7069636F2D73646B78
:10A4F8005C7372635C7270325F636F6D6D6F6E5CFC
:10A508007069636F5F666C6F61745C666C6F6174B1
:10A518005F696E69745F726F6D2E63005F5F61655E
:10A528006162695F666C6F61745F696E697400006F
:10A538004465627567000000626F6F74325F77323E
:10A548003571303830000000302E3100312E332E76
:10A55800310000007069636F000000004C6F67698C
:10A5680063416E616C797A65720000004A756E20ED
:10A57800323520323032320006005250BBFF3CB632
:10A588005CA50010060052503ABCA91150A5001055
:10A5980006005250E182887F40A500100600525004
:10A5A800D3F0754238A500106C656E203D3D203112
:10A5B80000000000463A5C5069636F53444B5C509E
:10A5C80069636F5C7069636F2D73646B5C7372632E
:10A5D8005C7270325F636F6D6D6F6E5C7069636F14
:10A5E8005F737464696F5C737464696F2E630000D1
:10A5F8007570646174655F75735F73696E63655FB9
:10A60800626F6F7400000000676574636861725F51
:10A6180074696D656F75745F757300000D0A0000CD
:10A62800E5630010E9630010F5630010456400104D
:10A6380029640010000000005553422073746469B7
:10A648006E202F207374646F7574000006005250DA
:10A6580053B4F4A140A600107570646174655F7509
:10A66800735F73696E63655F626F6F7400000000EB
:10A67800526173706265727279205069000000003F
:10A688005069636F00000000426F617264204344A8
:10A69800430000005265736574000000090254000D
:10A6A800030100807D080B0002020200000904007B
:10A6B8000001020200040524002001052401000114
:10A6C800042402020524060001070581030800107E
:10A6D80009040100020A0000000705020240000008
:10A6E800070582024000000904020000FF0001057E
:10A6F80012010002EF0201408A2E0A000001010245
:10A70800030100000000000078A6001088A60010D1
:10A718007C8E022090A600109CA60010282875693F
:10A728006E747074725F7420296E6578745F6275D8
:10A73800666665725F70747220262030623131312E
:10A748003131317529203D3D20300000463A5C50BA
:10A7580069636F53444B5C5069636F5C7069636FE6
:10A768002D73646B5C6C69625C74696E7975736275
:10A778005C7372635C706F727461626C655C726149
:10A788007370626572727970695C727032303430DD
:10A798005C6463645F7270323034302E6300000092
:10A7A80068775F646174615F6F6666736574286E4D
:10A7B8006578745F6275666665725F707472292069
:10A7C8003C3D205553425F445052414D5F4D4158E6
:10A7D80000000000556E68616E646C656420495223
:10A7E8005120307825780A007268706F7274203DA5
:10A7F8003D2030006463645F656470745F786665EB
:10A80800720000006463645F656470745F6F7065F4
:10A818006E0000006463645F7365745F61646472F2
:10A82800657373006463645F696E745F656E61620B
:10A838006C6500005F68775F656E64706F696E7441
:10A848005F616C6C6F6300006463645F696E697458
:10A858000000000021286275665F6374726C202610
:10A86800205553425F4255465F4354524C5F46550C
:10A878004C4C2900463A5C5069636F53444B5C501A
:10A8880069636F5C7069636F2D73646B5C6C69627C
:10A898005C74696E797573625C7372635C706F72F5
:10A8A8007461626C655C72617370626572727970F2
:10A8B800695C7270323034305C7270323034305FC0
:10A8C8007573622E630000006275665F6374726C54
:10A8D8002026205553425F4255465F4354524C5FF1
:10A8E80046554C4C000000006570202564202573F7
:10A8F8002077617320616C7265616479206176618B
:10A90800696C61626C6500005741524E3A2073745D
:10A91800617274696E67206E6577207472616E73F8
:10A92800666572206F6E20616C7265616479206162
:10A9380063746976652065702025642025730A0094
:10A9480043616E277420636F6E74696E7565207835
:10A95800666572206F6E20696E6163746976652022
:10A968006570202564202573000000006F75740051
:10A97800696E000073796E635F65705F6275666605
:10A988006572000025732025643A204153534552CF
:10A9980054204641494C45440D0A0000E47100101A
:10A9A8004271001072710010AE710010E471001055
:10A9B800E4710010CA71001072710010E471001087
:10A9C800E4710010E4710010E4710010E4710010EB
:10A9D800E4710010E471001054710010667A0010E0
:10A9E800407A00101C7C00101A7A00101C7C0010A1
:10A9F800827900100E7A00101C7C00109E790010DD
:10AA0800B6790010827C0010747C0010C67C00109F
:10AA1800367E0010B27D0010D27D0010DA7C001066
:10AA2800267D00103A7E0010757362645F6564705D
:10AA3800745F786665720000757362645F65647040
:10AA4800745F6F70656E0000757362645F6F706528
:10AA58006E5F656470745F70616972006F73616CBA
:10AA68005F71756575655F73656E640070726F639D
:10AA78006573735F6765745F646573637269707427
:10AA88006F72000070726F636573735F7365745FD4
:10AA9800636F6E666967000070726F636573735FDA
:10AAA800636F6E74726F6C5F726571756573740035
:10AAB8007475645F7461736B00000000D9820010C4
:10AAC80095830010D9830010D184001005860010EA
:10AAD80000000000757362645F636F6E74726F6C60
:10AAE8005F786665725F6362000000007475645F7A
:10AAF800636F6E74726F6C5F786665720000000039
:10AB0800636463645F786665725F63620000000077
:10AB1800636463645F6F70656E0000007475645FE2
:10AB28006364635F6E5F77726974655F666C757383
:10AB38006800000074755F656470745F76616C69A5
:10AB48006461746500000000747573625F696E6902
:10AB5800740000006C656E203E203000463A5C5060
:10AB680069636F53444B5C5069636F5C7069636FD2
:10AB78002D73646B5C7372635C7270325F636F6DAC
:10AB88006D6F6E5C7069636F5F756E697175655F17
:10AB980069645C756E697175655F69642E63000030
:10ABA8007069636F5F6765745F756E697175655FFE
:10ABB800626F6172645F69645F737472696E670063
:10ABC800666C6173685F6F666673202B20636F75B0
:10ABD8006E74203C3D205049434F5F464C415348DA
:10ABE8005F53495A455F425954455300463A5C50B1
:10ABF80069636F53444B5C5069636F5C7069636F42
:10AC08002D73646B5C7372635C7270325F636F6D1B
:10AC18006D6F6E5C68617264776172655F666C61A6
:10AC280073685C666C6173682E630000636F6E6E98
:10AC38006563745F696E7465726E616C5F666C6182
:10AC4800736820262620666C6173685F657869746E
:10AC58005F78697020262620666C6173685F726170
:10AC68006E67655F657261736520262620666C6174
:10AC780073685F666C7573685F636163686500001D
:10AC8800636F6E6E6563745F696E7465726E616C16
:10AC98005F666C61736820262620666C6173685F46
:10ACA800657869745F78697020262620666C617300
:10ACB800685F72616E67655F70726F6772616D2041
:10ACC800262620666C6173685F666C7573685F63BF
:10ACD8006163686500000000636F6E6E6563745F92
:10ACE800696E7465726E616C5F666C61736820264C
:10ACF8002620666C6173685F657869745F7869702F
:10AD080020262620666C6173685F666C7573685FC1
:10AD18006361636865000000666C6173685F646FF7
:10AD28005F636D64000000004E6F20444D41206356
:10AD380068616E6E656C7320617265206176616909
:10AD48006C61626C6500000070726F6772616D2DD6
:10AD58003E6C656E677468203C3D2050494F5F49E2
:10AD68004E535452554354494F4E5F434F554E54DA
:10AD780000000000463A5C5069636F53444B5C50D6
:10AD880069636F5C7069636F2D73646B5C73726366
:10AD98005C7270325F636F6D6D6F6E5C6861726458
:10ADA800776172655F70696F5C70696F2E63000010
:10ADB8004E6F2070726F6772616D2073706163658A
:10ADC800000000004E6F2050494F20737461746575
:10ADD800206D616368696E657320617265206176B4
:10ADE80061696C61626C650070726F6772616D5F3A
:10ADF8006D61736B203D3D20285F757365645F69E5
:10AE08006E737472756374696F6E5F737061636576
:10AE18005B70696F5F6765745F696E6465782870D9
:10AE2800696F295D20262070726F6772616D5F6D92
:10AE380061736B290000000070696F5F72656D6F48
:10AE480076655F70726F6772616D00005F70696F21
:10AE58005F66696E645F6F66667365745F666F725E
:0CAE68005F70726F6772616D0000000087
:10AE7400B4020010A80200109C02001080A500106B
:10AE8400900200108CA5001098A50010A4A5001035
:04AE940054A60010B0
:10AE980010B5D0231B0600241C570268EFF310815D
:10AEA80072B61368002BFCD0BFF35F8F0423C35620
:10AEB800002B08DB0368BFF35F8F00221A6081F361
:10AEC800108820BFE9E704710368BFF35F8F002291
:10AED8001A6081F3108810BD03000068EFF3108C2E
:10AEE80072B60268002AFCD0BFF35F8F04229A561C
:10AEF800002A0BDB002910D00A6000201B68BFF372
:10AF08005F8F00221A608CF310887047D0221206D7
:10AF1800127852B21A710120F0E70020EEE7000023
:10AF2800F8B5CE46474680B5040017009846036832
:10AF3800002B20D0D0231B061B785BB299462668CD
:10AF4800EFF3108C72B63568002DFCD0BFF35F8F1D
:10AF580004256557002D14DB2368BFF35F8F00229B
:10AF68001A608CF310883800414600F021F9002857
:10AF7800E5D000200FE00A4B0A4A7A210A4800F07F
:10AF88002FF94B4623712368BFF35F8F00221A60A5
:10AF98008CF310880120C0BCB946B046F8BDC04645
:10AFA8009C9B0010F49B0010649B0010F0B5C646F3
:10AFB80000B582B00700884600F002F904000D1EB3
:10AFC8001CDB0190FA22920000234046002100F089
:10AFD800FFF822002B0012184B419D4202D804D1E1
:10AFE800944202D901225242D317002B0CDB3800BD
:10AFF800FFF796FF02B080BCB846F0BD054B064A85
:10B008003F21064800F0ECF8024B034A3F21034871
:10B0180000F0E6F8449800100C9C001060980010AE
:10B0280010B50268EFF3108172B61368002BFCD0DC
:10B03800BFF35F8F0423C356002B0ADBFF23037182
:10B048000368BFF35F8F00221A6081F3108840BF46
:10B0580010BD034B034AA921034800F0C1F8C046BC
:10B06800B09B0010E89B0010649B0010094B1B78F4
:10B07800002B08D00CE09A00802149055118086877
:10B088000549505001333F2BF5DD024B01221A7060
:10B098007047C046928E0220D085022010B5024B20
:10B0A8000133984710BDC046D085022000280AD039
:10B0B80003231B02054A12685340C0229200134022
:10B0C800034A136070470223F3E7C0460C8001402F
:10B0D8000C900140F0B5D6464F464646C0B507002D
:10B0E8000E00150018239A461B88142290461088D3
:10B0F80028499847814653461B8842461088264966
:10B108009847040053461B884246108823499847AD
:10B1180080464B46002B0CD0002C0AD0002808D0C3
:10B12800FFF7A4FFC847A0470020FFF7BFFF2A008A
:10B138000FE01B4B1B4A80211B4800F051F8002BE5
:10B1480007D0002A05D0C0235B051B6E3370013A77
:10B1580001362B00134312D0C0235B059C6A0823D9
:10B168002340A107EBD5002DE9D0511B0D29E6D8C6
:10B178003878C02149050866013D0137DFE701201D
:10B18800FFF794FFC047FFF789FFE0BCBA46B14616
:10B19800A846F0BD49460000455800004643000057
:10B1A800E0AC001020AD0010F4AB00107047C046B2
:10B1B80001B40248844601BC604700BFA92D0010B5
:10B1C80001B40248844601BC604700BFCD2E001080
:10B1D80001B40248844601BC604700BFE95D001025
:10B1E80001B40248844601BC604700BFA93500107D
:10B1F8002804002009FF0000A080206000E007C0AC
:10B20800E0A04460A40001E00800000024810220BE
:10B21800200010005C0400200000000000800220D4
:10B2280004870220000000000000000014870220AC
:10B2380000000000000000001000000000000000F6
:10B2480000000100000000000000000000000200F3
:10B2580000000000000000000000030000000000E3
:10B26800000000000000FF000000000000B5486872
:10B2780001318E460047704609380149884700BDAC
:10B28800313C001000000000000000000000000039
:10B29800503300004C330000543300005233000098
:10B2A8004D5300004D430000533400004334000068
:10B2B8006565001000000000D56400100000000063
:10B2C8000001000074A9001078A90010F884022079
:10B2D80010000C000000E0FF1F000000000000004C
:10B2E8000000000000000000000000000000000056
:10B2F8000000000000000000000000000000000046
:10B3080005600010A9500010B9570010D55E001054
:08B31800ED020010E18E0010AF
:04000005100001E9FD
:00000001FF
